:100000000266BA3200000000000000026435000001
:1000100000000032000000000000000226E10000A5
:1000200067D90002331300000000000265010000E0
:1000300050523330324C434420763130362E352006
:100040004864773A462034303030752032392D30CC
:10005000332D30342031383A32302020D320202044
:10006000522045205320452054D250523330322064
:100070004C434420763130362E35002D2D2F2D2D3A
:10008000202D2D3A2D2D004350523A20004C6F6305
:100090003A20004C4F433A2000D22020202020203C
:1000A00020202020202020202020D200454E545205
:1000B0005920202000455849542020202000445534
:1000C0005459204558495400494E5445524E414CCC
:1000D00000D120202020202020202020202020208F
:1000E0002020D1435243202020204520722072201E
:1000F0006F20720020202020200020D1466C6173E8
:100100006820435243204572726F722000D3436FC0
:100110006E666967204D656D204572726F7200D3FF
:100120002053657276696365204F4E00D320536576
:100130007276696365204F464600D2204D41535484
:100140004552204944203D20203F2000D353657470
:100150002074696D652048484D4D202020D200D381
:10016000536574206461746520524D4D444457209A
:10017000D200D2202020202020202020202020203B
:10018000202020D2D501055245473A200000D3D582
:10019000021044206F2077206E206C206F20612099
:1001A000642000D12020202020202020202020207A
:1001B0002020202020D1D5030C50617373776F72FB
:1001C000643F203A2000D2D5041020416363657358
:1001D000732064656E696564202000D2D505102007
:1001E000416363657373206772616E746564200098
:1001F000D1D50410204163636573732064656E6913
:1002000065642020D2D50610204E6F204475616CA5
:1002100020456E747279202000D3D5091044756191
:100220006C20456E747279204D6F64652000D1D5C5
:100230000A0A2020204572726F722023002020209D
:100240002000D1D50C10202020415042205265734F
:1002500065742020202000D2D50E104C696D697481
:10026000206578636565646564202000D50F0C4EB9
:100270004F524D414C20202020202000D1D5041089
:1002800020204143434553532044454E59202020CC
:10029000D2D51010204150422056696F6C617469AC
:1002A0006F6E202000D1D50D1020202020496465DC
:1002B0006E74204F4B20202020D2D51010204150AA
:1002C000422056696F6C6174696F6E202000D2D530
:1002D0001110204E6F206F6E6520696E7369646522
:1002E000202000D1D512102020205573657220499E
:1002F00044203D203F202000D320202020552053A3
:1003000020452052D2D51610202050726F6772619E
:100310006D6D696E6700D3202020494E5354414CC7
:100320004C455220202020D2D51610202050726F2C
:100330006772616D6D696E6720202000D2202020D9
:100340002046205220452045202020202000D22079
:10035000202045205820492053205420532020009D
:10036000D1D5041020204143434553532044454EEA
:1003700059202020D2D506102020496E7075742097
:10038000426C6F636B73202000D1D5041020204194
:1003900043434553532044454E59202020D2D5078E
:1003A000102020434C4F534544204D4F44452020BE
:1003B0002000D1D50410202041434345535320440D
:1003C000454E59202020D2D508104F7574206F66F5
:1003D0002074696D65207A6F6E6500D1D504102098
:1003E000204143434553532044454E59202020D2B9
:1003F000D50B10204F464620636F6E646974696F99
:100400006E202000D1D51310202053574954434863
:100410002044454E59202020D2D508104F75742015
:100420006F662074696D65207A6F6E6500D1D504A2
:100430001020204143434553532044454E5920202A
:1004400020D2D5141020202020505245414C41523A
:100450004D2020202000D1D51510205377697463DA
:100460006865722049443D203F2000C28E53890FA9
:10047000438910758BD6758D97C28FD28E308FFDC4
:10048000C28E22C28E53890F438910758BEB758DF6
:10049000CBC28FD28E308FFDC28E22C28E53890F77
:1004A000438910E58AC4242BF58B758DEBC28FD25E
:1004B0008E308FFDC28E22F9C3137004A2588018AB
:1004C00014C0E0030303540F243DF8D0E0540704A4
:1004D000F5F0E213D5F0FCE992E02275F006120582
:1004E0008B22C2A075F00612058BD2A0221204E264
:1004F0001204DB1204E21204DB1204E21204DB1227
:1005000004E21204DB1204E275F01812058B22C219
:10051000A075F04B12058BD2A022755B041232E15C
:10052000C2A075F0C812058BD2A022755B051232ED
:10053000E112050F75F01E12058B12050F22755B77
:10054000071232E11204F922755B061232E112043D
:10055000FF221204ED1204ED22755B071232E175E1
:100560005B061232E11204FF1204FF1204FF22D2D2
:1005700008C26D1204E275F01212058BC208C26D3A
:10058000221204E275F01212058B2212046B20284D
:1005900007C0F01228FAD0F0D5F0F0227004A2586B
:1005A000B322C0E0141205ABD0E022C0E003030385
:1005B000540F28F8D0E0C0E0540704F5F0E213D55A
:1005C000F0FCD0E0221204ED75F01412046BD5F0AB
:1005D000FA221204F975F0C812046BD5F0FA80F211
:1005E00022C0F075F0DCD5F008B203121818125DC5
:1005F0003AC0F0120873D0F030E7EBD0F022AAF046
:100600001205E1E5336530F5F0E534653145F0601C
:100610000C1207588530338531341205E112082653
:100620001205E112085A1205E112076B8AF022AA9C
:10063000F01205E1E5336530F5F0E534653145F05C
:10064000600C1207588530338531341205E11208E9
:100650000C1205E112085A1205E112076B8AF0220A
:1006600079207530017531037532E090007B1205F9
:10067000E11207581205E11207D4790075300175AF
:10068000310475320090009B1205E11207581205E3
:10069000E11207D479E075300175310575320090AB
:1006A000019B1205E11207581205E11207D48530AB
:1006B0003385313422AAF01205E1E5336530F5F0D7
:1006C000E534653145F0600C1207588530338531CB
:1006D000341205E11207B68AF022AAF01205E1E50C
:1006E000336530F5F0E534653145F0600C1207589C
:1006F0008530338531341205E11207988AF022C023
:10070000F075F00833C29792A600D297D5F0F5D0D5
:10071000F022C0F075F008C297D29700A2A133D59D
:10072000F0F5D0F022D204D297D2A6D2A1D20512EF
:10073000181822E53133E5303322C3E5313322E5A1
:1007400032221206FF1207331206FF12073A120670
:10075000FF12073F1206FF22120725C205121818C2
:100760007453120742D20512181822120725C20527
:100770001218187458120742D205121818221207BC
:1007800025C2051218187454120742E41206FF120B
:100790000712D20512181822120725C205121818BE
:1007A0007454120742E41206FF120712F608D9F930
:1007B000D20512181822120725C2051218187454EF
:1007C000120742E41206FF120712F208D9F9D20505
:1007D00012181822120725C205121818745412078D
:1007E00042E41206FF120712F0A3D9F9D20512183B
:1007F0001822120725C0E0C20512181874841207C7
:1008000042D0E01206FFD20512181822120725C2A4
:10081000051218187484120742E61206FF08D9F967
:10082000D20512181822120725C20512181874844E
:10083000120742E21206FF08D9F9D205121818224F
:10084000120725C2051218187484120742E0120616
:10085000FFA3D9F9D20512181822120725C20512D2
:1008600018187483120742D20512181812046B125A
:10087000046B22C20512181874571206FF120712D1
:10088000D20512181822D2A6D2A1D297D204D2052C
:10089000121818B20312181875F00212046BD5F072
:1008A000FAC204B20312181875F00212046BD5F0E4
:1008B000FAD204B203121818227530017531DB75B3
:1008C00032001205E1120B5A7533FF7534FF22AE68
:1008D00083AD8290DB007F207404F9747CF875305E
:1008E000018583318582321206DA787CE66E7025C6
:1008F00008E66D702008E6601AB4FF0280131674D3
:1009000004F9747CF87530018583318582321206D2
:100910002FC322D322A3A3A3A3DFBD80F490DB00C7
:100920007F207404F9747CF87530018583318582E9
:10093000321206DA787CE66E700908E66D700408FB
:10094000E6FC22A3A3A3A3DF0A7CFF2290DB007FA7
:10095000207BFF7404F9747CF87530018583318540
:1009600082321206DA787CE66E702C08E66D70270B
:1009700008ECB4FF0D787C76FF0876FF0876FF0858
:1009800074FFF67404F9747CF87530018583318541
:10099000823212062FC322BBFF10787CE6B4FF0A16
:1009A00008E6B4FF05C374209FFBA3A3A3A3DFA3A2
:1009B000BBFF02D322EB232354FC2400F582758372
:1009C000DB50020583787CEEF608EDF608ECF608BD
:1009D000E4F67404F9747CF87530018583318582FE
:1009E0003212062FC32275830075F08E7530028592
:1009F0008331753200C0F0C0831205E1120B5AD06A
:100A0000830583D0F0D5F0E475830075F0DA753096
:100A100003858331753200C0F0C0831205E1120BEB
:100A20005AD0830583D0F0D5F0E47533FF7534FFD9
:100A30002275830075820075F08EC0F0C082C0837D
:100A40007530028583317532001205E1120758D0E6
:100A500083D082C082C083753000858231753200B8
:100A60001205E112085AD083D08205830582D0F0A6
:100A7000D5F0C775830075820075F0DAC0F0C082CA
:100A8000C0837530038583317532001205E112078A
:100A900058D083D082C082C0837530018582317581
:100AA00032001205E112085AD083D08205830582F4
:100AB000D0F0D5F0C77533FF7534FF22758300750C
:100AC000820075F08EC0F0C082C0837530008583CF
:100AD000317532001205E1120758D083D082C082EE
:100AE000C0837530028582317532001205E112082B
:100AF0005AD083D08205830582D0F0D5F0C77583A4
:100B00000075820075F0DAC0F0C082C083753001D4
:100B10008583317532001205E1120758D083D082E7
:100B2000C082C0837530038582317532001205E1C1
:100B300012085AD083D08205830582D0F0D5F0C741
:100B40007533FF7534FF22120725C2051218187479
:100B500050120742D20512181822120725C2051298
:100B600018187481120742D205121818221207258C
:100B7000C2051218187484120742E81206FFD9FA47
:100B8000D20512181822AAF01205E1E5336530F5F6
:100B9000F0E534653145F0600C1207588530338537
:100BA00031341205E1120B6D1205E112085A8AF078
:100BB00022120725C2051218187454120742E412B3
:100BC00006FFE4C0E0120712D0F025F0D9F5D205F7
:100BD00012181822758300758202800675830075CD
:100BE0008200E475F08D858230858331753200C0D6
:100BF00082C083C0F0C0E01205E11207581205E17F
:100C00007900120BB1D0F025F0D0F0D083D082055E
:100C100083D5F0D2858230858331753200C0E012F1
:100C200005E11207581205E17920120BB1D0F02529
:100C3000F07533FF7534FF227583007582038006DB
:100C4000758300758201E475F0DA85823085833121
:100C5000753200C082C083C0F0C0E01205E1120707
:100C6000581205E17900120BB1D0F025F0D0F0D088
:100C700083D0820583D5F0D27533FF7534FF05E04C
:100C80002275830075F00075300085833175320060
:100C9000C0F0C0831205E1120B5AD0830583D0F057
:100CA000D5F0E47533FF7534FF75830075F0DA75A0
:100CB0003001858331753200C0F0C0831205E11226
:100CC0000B5AD0830583D0F0D5F0E47533FF75342B
:100CD000FF221205057556FA3090FA75F0051204D8
:100CE0006BD5F0FA7556FA2090FA22E578B406FA38
:100CF000C083C082C0E074D1126A6ED0E0D082D0CE
:100D000083C083C082C0E07428126A6ED0E0D082B3
:100D1000D083E5831257AAE5821257AAC083C08206
:100D2000C0E07429126A6ED0E0D082D0837800E2ED
:100D30001257AAC083C082C0E0742F126A6ED0E03E
:100D4000D082D0837801E21257AAC083C082C0E06B
:100D50007420126A6ED0E0D082D083C083C082C07B
:100D6000E0743E126A6ED0E0D082D083C083C0822D
:100D7000C0E07420126A6ED0E0D082D0837802E2A4
:100D80001257AA120CD222C0E0E578B4096AC083D7
:100D9000C082C0E074D3126A6ED0E0D082D083D01B
:100DA000E0C083C082C0E0126A6ED0E0D082D083FF
:100DB000C083C082C0E0743A126A6ED0E0D082D0A4
:100DC00083C083C082C0E07420126A6ED0E0D082FB
:100DD000D083787CE61257AA08E61257AA08E612D2
:100DE00057AA08E61257AA08E61257AA08E61257A9
:100DF000AAD2AF120CD2C0E0D0E022E578B40570E0
:100E0000ED600F1414600B146008146005ED248865
:100E1000505EC083C082C0E074D3126A6ED0E0D04E
:100E200082D083E583C0821257AAD082E58212570E
:100E3000AAC083C082C0E0742F126A6ED0E0D08254
:100E4000D083ED1257AAC083C082C0E07420126A1A
:100E50006ED0E0D082D083787CE61257AA08E612E2
:100E600057AA08E61257AA08E61257AA08120CD287
:100E70002222E578B405F9ED248850F4C082C083BD
:100E8000C083C082C0E074D2126A6ED0E0D082D03B
:100E900083787CE60354012430C083C082C0E01212
:100EA0006A6ED0E0D082D083C083C082C0E0743A42
:100EB000126A6ED0E0D082D083E61257AA08E612FA
:100EC00057AAC083C082C0E07420126A6ED0E0D0FE
:100ED00082D083C083C082C0E0743E126A6ED0E0CC
:100EE000D082D083D083D082E583C082C083125762
:100EF000AAD083D082E582C082C0831257AA120C86
:100F0000D2D083D0822222E578B40540ED248850E7
:100F10003BC083C082C0E07420126A6ED0E0D082F1
:100F2000D083C083C082C0E0743A126A6ED0E0D031
:100F300082D08374303078027431C083C082C0E0C4
:100F4000126A6ED0E0D082D083120CD222301359B4
:100F50007881E6540FC0E0E6C4540375F00AA4D0CB
:100F6000F025F0FD7882E630E402240A540FFE906A
:100F70001A007F3C7404F97400F8753001858331E0
:100F80008582321206B57800E26D701708E26E7045
:100F90001208E2C42354E0F5F07882E6541F45F0CD
:100FA000F68006A3A3A3A3DFCB2212690C120F4D78
:100FB00012691BFEAFF01260867DFF0DED30E70178
:100FC00022D27875F004A4247BF582E5F03400F594
:100FD00083C082C083787CE0F6A308E0F6A308E033
:100FE000F6A308E0F6D083D082120DFB787C8683CE
:100FF000088682787CB6FF0708B6FF03021063C339
:10100000E58233F582E58333F583E58224E0F582DA
:10101000E5833405F583787EE6704808E66044FB96
:101020007402F9747CF8753001858331858232123F
:1010300006DA120E71A3A3787CE60856B4FF030209
:101040001063787C86F053F07F08E6C39EC0E0E52D
:10105000F09FD0F0400445F07009787CE6A2E7925A
:1010600078DBBD120F06BD003DB278122EED403385
:1010700020413020290E30420B2057053078248043
:101080000320781FA278925792E0A25892E1F5F0DF
:1010900013925865F030E00B205805122F7D800325
:1010A000122F8C020FBBED14C0E0030303540F2476
:1010B0003DF8D0E0540704FB7400D333DBFD3078F7
:1010C00005FBE24B8004F4FBE25BF2020FBB12066D
:1010D000FF1207331206FF12073AD2E01206FF1280
:1010E000073F1206FF22120725C205121818745472
:1010F0001210CEE41206FF120712F608D9F9D20533
:1011000012181822120725C205121818748412101A
:10111000CEE61206FF08D9F9D2051218182290FC63
:1011200000753004753100753200C082C083755679
:10113000FA1205E112075885307A853179790878F5
:101140007C1205E11210E612131AD083D08270448B
:10115000C082C083788086830886821211CB4024A7
:10116000787E86830886821211CB40181211EAE538
:1011700082600AE576B5790CE577B57A07D083D039
:10118000820211A6787EE6249AF612135D12572C7D
:10119000D083D0820531E53170020530A3E5824568
:1011A0008370871211AD7533FF7534FF22787E7618
:1011B00000087600788076000876000876000876C9
:1011C00000757A0475790012133922C082C083E554
:1011D000822400F582E5833480F5834005D083D0F6
:1011E0008222D083D08290000022E58275F008A48C
:1011F000F582E5F0C58375F008A42583F583E5F055
:101200003404F577E5822400F582E5833400F58324
:10121000500205778583762212573CD083D08222F4
:10122000C082C0831212F370EF787E8683088682B4
:101230001211CB40E31211EA121667787C7600781F
:1012400080E518F608E519F60876000876007408B7
:10125000F9747CF885773085833185823212062FC8
:101260007404F97480F88577308583318582321271
:1012700006DA75F004787C7980E667600280990868
:1012800009D5F0F51212FA787E8683088682A312B9
:1012900011CB787EA68308A6827880868308868212
:1012A0001211CB787EE66583700A08E665827004C9
:1012B000A31211CB7880A68308A682C07AC0798554
:1012C000777A857679121339D0E0D0F0B57909C5EF
:1012D000F0B57A028018C5F0C07AC07985F07AF549
:1012E00079787EE62499F612135DD079D07AD0838E
:1012F000D082221212FA12131A22857A308579319D
:101300007532001205E11207587908787C1205E160
:101310001210E6853033853134227881E61826189C
:1013200026182618245566700F7881E61866186608
:1013300018661866186499662212134012135D220B
:101340007881E6182618261826182455F67881E69E
:101350001866186618661866186499F622857A3039
:101360008579317532001205E11207581205E179CD
:1013700008787C1211041205E112085A1205E112D4
:10138000076B853033853134221212F37030787E4A
:10139000E6C0E008E6C0E0088683088682C3D0E0A5
:1013A0009582F582D0E09583F58350104582600CDC
:1013B000E5822400F582E5833480F583C322900022
:1013C00000D322C2B6121389E433C0E0753800742A
:1013D000031240B6E51E1240B6E51F1240B6745324
:1013E0001240B6D0E01240B674001240B67400123B
:1013F00040B6E5831240B6E5821240B6E5381240A9
:10140000B63099FD22C2B6E5366004F4FF8004FFD1
:101410001211AD75380074031240B6E51E1240B6C5
:10142000E51F1240B674561240B6EF1240B6E538CA
:101430001240B63099FD227401C0E0787C75F00846
:10144000E4F608D5F0FBD0E0D32212138940E8601F
:10145000E87880868308868212145DC322C082C029
:1014600083E58275F008A4F582E5F0C58375F00880
:10147000A42583F583E5F03404F577E5822400F5AF
:1014800082E5833400F583500205777408F9747C93
:10149000F88577308583318582321206DAD083D0A1
:1014A00082221213897F0850051211AD7F00787EC9
:1014B0008664088665088666088667C2B675380041
:1014C00074031240B6E51E1240B6E51F1240B67412
:1014D000541240B6E5361240B6EF1240B6E536601B
:1014E0003CE5676565F5F0E566656445F0600B858C
:1014F000678285668312145D8003121439856782C2
:10150000856683A31211CB858267858366787C7597
:10151000F008E61240B608D5F0F8D536C4E5381222
:1015200040B63099FDC322E5367007C2AF12138969
:101530005005E536F4800C7880A66608A66712137D
:1015400039E536D2AFC0E0C2B67538007403124038
:10155000B6E51E1240B6E51F1240B674551240B6ED
:10156000D0E01240B6E5381240B63099FDD322C221
:10157000B612690C75380074031240B6E51E1240AD
:10158000B6E51F1240B674571240B67881E62323A1
:1015900054031240B67882E630E402240A541F1243
:1015A00040B67881E6C45401F5F0A4E5F0E6540FA6
:1015B00025F01240B67881E6C45401F5F0A4E5F0B8
:1015C000E6540F25F01240B6787FE6C45403F5F0D8
:1015D000A4E5F0E6540F25F01240B6787EE6C45438
:1015E00003F5F0A4E5F0E6540F25F01240B678823A
:1015F000E603C454071240B6E5381240B63099FDF0
:10160000D322C2B675380074031240B6E51E1240EC
:10161000B6E51F1240B674581240B6742023235406
:10162000FC041240B674201240B690DB007F207498
:1016300004F9747CF8753001858331858232120695
:10164000DA787CE61240B608E61240B608E61240A8
:10165000B608E61240B608A3A3A3A3DFD2E538126A
:1016600040B63099FDD32212690C7882E630E4024C
:10167000240A540FC4F97881E6C4540375F00AA40F
:10168000F5F0E6540F25F0C31349787DF67881E62E
:1016900092E754C0F9787FE6C4540775F00AA4F5C0
:1016A000F0E6540F25F049F97880E6C4540375F04C
:1016B0000AA4F5F0E6540F25F0F5F0787EE65470B4
:1016C0002345F0787FF6787EE9F622C082C083C099
:1016D00083C082C0E074D2126A6ED0E0D082D08320
:1016E000E5301257AAE5311257AAC083C082C0E084
:1016F0007420126A6ED0E0D082D083C083C082C0D2
:10170000E07468126A6ED0E0D082D083787EE612F0
:1017100057AA08E61257AAC083C082C0E0742012FC
:101720006A6ED0E0D082D083C083C082C0E074747F
:10173000126A6ED0E0D082D08308E61257AA08E67B
:101740001257AAC083C082C0E07420126A6ED0E033
:10175000D082D083C083C082C0E07420126A6ED071
:10176000E0D082D083C083C082C0E07420126A6E51
:10177000D0E0D082D083C083C082C0E07420126ADF
:101780006ED0E0D082D083120CD2D083D08222538C
:10179000630F53620F5318F053190FC2AFE5622362
:1017A00024ADF8E5184519F608A61A056253620F2C
:1017B000E562B56305056353630FD2AF22E563B5F8
:1017C00062057400780022C33324ADF8E6C0E00857
:1017D000E6F8D0E02275F0083392A3D2A2C2A2D5D7
:1017E000F0F622E51DA2E3B3306B029206306E02E2
:1017F0009209306D029208A20692E0A20792E1A23D
:101800000992E2A20892E3A20A92E4A20C92E5A253
:101810000B92E6A20192E722A2AFC2AFC0D0C0E015
:10182000C0F0C2A4C2A2C2A3E561A20292E4A204D3
:1018300092E5A20592E6A20392E71217D5E560129F
:1018400017D51217E31217D5D2A4C2A4D0F0D0E056
:10185000D0D092AF2230590122756100756000121C
:10186000181820A54C7560FE7561FF7A0C121818C7
:1018700030A50DD3E56033F560E56133F561DAED50
:10188000EA602E15E0606615E0602B15E0605915E2
:10189000E0605015E0604715E0603E15E0603515EA
:1018A000E0602C15E0602315E0601A15E0601180FF
:1018B0000A74FF0218F874000218F874010218F88C
:1018C00074020218F874030218F874040218F87409
:1018D000050218F874060218F874070218F874085C
:1018E0000218F874090218F8740A0218F8740B0246
:1018F00018F8F54475450122B544F7D545F9B4FF0C
:101900000280F4D259F54680EE3059FDC2A075F040
:101910000612058BD2A075F01412058BE546C2594C
:10192000223028037555F012257A205907740F309C
:10193000280580F312190922F5F00303543FB4027D
:1019400067E53F64086005E53FB40D59E5F089F0AF
:10195000C0F030131CC0E07871E26013C33350054F
:10196000D0E00219841204B750F6D0E0021971D009
:10197000E0D0F0A9F05403B40211C23BA23BB392F1
:101980000B021A12D0F0A9F0021A12B4010AD23BCB
:10199000A23BB3920B021A12B4030AB23BA23BB3AE
:1019A000920B021A12021A10B40365E54064086033
:1019B00005E540B40DEFE5F089F0C0F030131CC030
:1019C000E07872E26013C3335005D0E00219EE12E2
:1019D00004B750F6D0E00219DBD0E0D0F0A9F05403
:1019E00003B40211C23CA23CB3920C021A12D0F012
:1019F000A9F0021A12B4010AD23CA23CB3920C0222
:101A00001A12B40309B23CA23CB3920C80048000C9
:101A1000D322C322786D75F00EE4F208D5F0FB7482
:101A2000FF7875F27876F222D24E6F206578746571
:101A30006E6465642020202020202020007570FF27
:101A4000121A14C213C212120C40602E20132A74F0
:101A500001F9747CF875300075318C7532EE120620
:101A6000DA797CE7B4FF12C24BC24CC24DC24EC2FF
:101A70004FC250C251C252C253221206607401F9C1
:101A80007470F87530017531037532A01206DA747E
:101A90000EF9746DF87530017531037532A11206B7
:101AA000B57410F9744DF87530017531037532C095
:101AB0001206B57410F9745DF8753001753103754F
:101AC00032D01206B5D213D21222797C774609772A
:101AD0004C09776A0977A07404F9747CF8753000B2
:101AE00075318D75322012062F7404F9747CF875E7
:101AF000300275318D75322012062F22E4A22E920B
:101B0000E0A22F92E1A23092E2797CF77401F9749D
:101B10007CF875300075318C7532E812062F22740E
:101B200001F9747CF875300075318C7532E8120655
:101B3000DA797CE7A2E0922EA2E1922FA2E2923023
:101B400022797CE4A23D92E0A23E92E1A23F92E2A1
:101B5000A22592E392E492E5A24192E6A24292E7A4
:101B6000F709E4A24092E0A24392E1A24492E2A2E9
:101B70004592E3A24792E4A24892E5A24992E6A2E6
:101B80004A92E7F709E4A24B92E0A24C92E1A24DFF
:101B900092E2A24E92E3A24F92E4A25092E5A251A9
:101BA00092E6A25292E7F7E4A25392E0F77404F9A6
:101BB000747CF875300075318C7532EC12062F226A
:101BC0007404F9747CF875300075318C7532EC1240
:101BD00006DA797CE7A2E0923DA2E1923EA2E2928F
:101BE0003FA2E39225A2E69241A2E7924209E7A230
:101BF000E09240A2E19243A2E29244A2E39245A283
:101C0000E49247A2E59248A2E69249A2E7924A09E5
:101C1000E7A2E0924BA2E1924CA2E2924DA2E392A3
:101C20004EA2E4924FA2E59250A2E69251A2E79210
:101C30005209E7A2E0925322797CF77401F9747C8F
:101C4000F875300075318C7532E412062F2274015C
:101C5000F9747CF875300075318C7532E41206DA4F
:101C6000797CE7227401F97439F875300075318C8C
:101C70007532FC12062F227401F97439F8753000A0
:101C800075318C7532FC1206DA227401F9743AF857
:101C900075300075318D75320012062F227401F9EE
:101CA000743AF875300075318D7532001206DA22FB
:101CB0007402F97439F875300075318C7532FD1283
:101CC00006B57402F9743BF875300075318D7532C4
:101CD000011206B5227402F97439F87530007531B5
:101CE0008C7532FD1205FE7402F9743BF8753000F4
:101CF00075318D7532011205FE227401F9743BF8BD
:101D000075300075318C7532F012062F7401F9743C
:101D10003CF875300075318C7532F412062F740161
:101D2000F9743DF875300075318C7532F612062F56
:101D3000227401F9743BF875300075318C7532F0FE
:101D40001206DA7401F9743CF875300075318C753F
:101D500032F41206DA7401F9743DF8753000753109
:101D60008C7532F61206DA7401F9743EF87530009B
:101D700075318C7532F21206DA227401F9743FF86B
:101D800075300075318C7532F812062F7401F974B4
:101D900040F875300075318C7532FA12062F7401D7
:101DA000F97441F875300075318C7532FB12062FCD
:101DB000227401F9743FF875300075318C7532F872
:101DC0001206DA7401F97440F875300075318C75BB
:101DD00032FA1206DA7401F97441F875300075317F
:101DE0008C7532FB1206DA227402F9741EF8753013
:101DF0000075318C7532E012062F227402F9741EC0
:101E0000F875300075318C7532E01206DA22C08226
:101E1000C083E58275F008A42420F582500205F005
:101E2000A8F0E58375F008A4282400F583787C7673
:101E3000FF7401F9747CF875300085833185823236
:101E400012062FA3A3A3A3A37401F9747CF8753021
:101E50000085833185823212062FD083D082C21250
:101E6000220809E7C4F5F066540F700D08E7F5F095
:101E700066540F7004DAEAE422E6540FC5F0540FFA
:101E8000C395F09211740122788179277A03E6C410
:101E9000540FF309E6540FF30908DAF2792778A012
:101EA0007A06E6540FF6E36670080908DAF4E4C22D
:101EB0005F22792C78A57A06C3E3961918DAFA928C
:101EC00011792C78A57A06E3540FB40F08E6540F65
:101ED000B40F108008E6540FB40F0B80061819DAFF
:101EE000E680CB740122C3E396B409028012146029
:101EF0000FC3E3F5F0E695F0B4090280031470E334
:101F0000E9B42704E4D25F221918E366540F60F0A5
:101F100080D1121E88701A305F1720401575185036
:101F200085831985821A12178F7554B4D25BD25EDD
:101F3000E42204227408F9747CF875300075318C41
:101F40007532C01206DA7894797C7A05121E632203
:101F50007408F9747CF875300075318C7532C012D4
:101F600006DA121F12227405F9747CF875300075B8
:101F7000318C7532C012062F227403F97481F87502
:101F8000300075318C7532C512062F22C082C08395
:101F9000E5822420F582E583347DF5837401F974AC
:101FA00042F87530008583318582321206DAD0839B
:101FB000D082C082C083E58275F008A42420F58217
:101FC000500205F0A8F0E58375F008A4282400F578
:101FD000837408F9747CF87530008583318582320A
:101FE0001206DAD083D08222C082C083E58275F0E7
:101FF00008A42420F582500205F0A8F0E58375F0CE
:1020000008A4282400F5837408F97494F875300046
:102010008583318582321206DAD083D08222C08253
:10202000C083E58275F008A42420F582500205F0F3
:10203000A8F0E58375F008A4282400F5837406F958
:10204000747CF87530008583318582321206DAD0CF
:1020500083D082227405F9747CF8753000753100E4
:102060007532201206DA7894797C7A05121E632282
:10207000751B20751C009000007405F9747CF875C0
:102080003000851C31851B321206DA7894797C7A0F
:1020900005121E636018E51B2408F51B5002051C81
:1020A000A3E583B40FD3E582B4A0CE740122121F3E
:1020B0008CE42220120280B8751B00751C00757418
:1020C0009F75750FE574251BC2E0F582E575351C1B
:1020D000F583C082C083E5822400F582E583341B4A
:1020E000F5837402F9747CF875300185833185823B
:1020F000321206DA787C8683088682121F8C7894E6
:10210000797C7A05121E637005D0F0D0F022D0835E
:10211000D082C3E58313F583E58213F58220111481
:10212000E58245836023E58224FFF574E58334FF6F
:10213000F5758007A385821B85831CC3E574951BF9
:10214000E575951C40030220C4740122751B25759A
:102150001C009000007403F97481F8753000851C30
:1021600031851B321206DA121F126018E51B240893
:10217000F51B5002051CA3E583B40FD9E582B4A07A
:10218000D4740122121F8CE42278A0E6540FB40FFD
:102190000302222320120280B3751B00751C0075F8
:1021A000749F75750FE574251BC2E0F582E57535E2
:1021B0001CF583C082C083E5822400F582E5833468
:1021C0003BF5837402F9747CF875300185833185A1
:1021D00082321206DA787C8683088682121F8C127D
:1021E0001F127005D0F0D0F022D083D082C3E583D7
:1021F00013F583E58213F582201114E5824583608F
:1022000022E58224FFF574E58334FFF5758007A38A
:1022100085821B85831CC3E574951BE575951C4061
:1022200002808274012278947A0579A8E6540FC45A
:10223000F5F008E6540F45F0F70809DAEF22D20668
:10224000C26BD209C26ED208C26DD2A075F0021262
:10225000046BD5F0FA20A047C0E0EAC0E0C083C01C
:102260008290005C126ACAD082D083D0E0AAE0D00B
:10227000E0D228C206C26BD209D26EC208C26DC2B9
:1022800007C26C120505B20312181875F00F12047C
:102290006BD5F0FA30A0EC122313C2AF02669BD2CA
:1022A000A0120BDC70071222DA121A3D22C2287526
:1022B00056FA75F06412046BD5F0FAC2A0D209C2C6
:1022C0006E75F06412046BD5F0FAD2A0C209C26E2A
:1022D000D2A012048330A08080D3121B1F121BC017
:1022E000121C4EA2E09254A2E19255A2E292561222
:1022F0001C77121C9D121D31121DB1121CB0121D33
:10230000FB22D206C26BD209C26ED208C26DC207CE
:10231000C26C22D2281255CD40E8D206C26BD20937
:10232000C26ED208C26DC207C26CC01EC01F787CCC
:102330009000007A08E6F008A3DAFA122368787CA5
:102340009000007A08E0F608A3DAFA900000124E36
:102350008A121F66121F79D01FD01E121DE8124F5D
:10236000041211AD1208B922120C81751E30751FAE
:1023700030C22EC22FC230C23DC23EC23FC225C2B1
:1023800041C242C240D243C244C245C247C248C20F
:1023900049C24AC24BC24CC24DC24EC24FC250C2C9
:1023A00051C252C25378397422F2087400F2783B59
:1023B0007406F2087400F2C254C255C2567539044C
:1023C000753A09753B01753C02753D04753E04750F
:1023D0003F07754000754100121DE8121AFC121BE0
:1023E00041C2E0A25492E0A25592E1A25692E212BA
:1023F0001C38121C64121C8A121CFA121D7A121C40
:10240000D5C213C212121ACA12626922302616C22B
:1024100026C2AC12049B12049BD2991224D6C26528
:10242000D2B612650C301C16C21CC2AC12049B1230
:10243000049BD2991214A2C265D2B612650C301E4A
:1024400016C21EC2AC12049B12049BD2991215270D
:10245000C265D2B612650C301D16C21DC2AC120484
:102460009B12049BD2991213C3C265D2B612650C9B
:10247000301F16C21FC2AC12049B12049BD29912C9
:102480001405C265D2B612650C302016C220C2AC4B
:1024900012049B12049BD29912156FC265D2B61218
:1024A000650C302116C221C2AC12049B12049BD2CF
:1024B00099121602C265D2B612650CE57B6013B4A0
:1024C0000105122F5F8008B40205122F6E8000757F
:1024D0007B001228FA22126383C2B6753800740397
:1024E0001240B6E51E1240B6E51F1240B6745012F7
:1024F00040B6747D1240B6900000E536600F900340
:10250000E81460099007D0146003900BB87E7D7FBB
:102510000875F000C0F012637EB40203D38001C3DB
:10252000D0E033F5F0A3DFEC1240B6DEE2E538127E
:1025300040B63099FD22307004C270800975F00CED
:1025400020B305D5F0FAD322C32220512C2028290C
:1025500012253650241226B6E8C0E0E9C0E0EAC0F1
:10256000E0755B0075F00312046BD5F0FA1231844C
:10257000D0E0FAD0E0F9D0E0F822D2688008C26852
:102580001225EE754300C227D2707556FA7440309A
:102590002802740CF553C267C259E553603B1225FB
:1025A0004A20673575F00312046BD5F0FA12240C3B
:1025B00020280320271A3059E1D27720681B755351
:1025C00060121909B40B0D75F00812046BD5F0FAFE
:1025D000D26780051225E180C1C266D2AF7556FA76
:1025E00022534307F8E54324A0C8F605432278A008
:1025F00075F00874FFF608D5F0FB22306609202D2F
:1026000003D22D22C26622C22D22D297122614C2D4
:102610009712261422C297C2B5122614D2971226F8
:1026200014D2B5122614C29712261475F0083392EC
:10263000B512260AD5F0F722D2B775F008D2971254
:102640002614A2B7C29712261433D5F0F022C297EF
:10265000C2B5122614D297122614D2B5122614C26D
:1026600097122614D2B512260A12260A12260A2218
:10267000D297D2B77473122615744B122615745064
:1026800012261512049B74081226151226382324CC
:102690003F3019022420543F4480122615746B12D7
:1026A0002615120483746812261512049B74601296
:1026B000261512264E22C2ABC28ED2AFD297D2B707
:1026C00022C2AFC28E53890F438910758B19758D45
:1026D000FCC28FD28ED2AFC263D2BBD2AB3063FD0D
:1026E00022C0D0A2B79262D263D0D0C2ABC28EC297
:1026F0008F758B0D758DFED28EC2AF32D26880047D
:10270000D270C268C2277556FAD22C7440302802A3
:10271000740CF5531225EE754300C267C266C259A8
:10272000C26A12240C202803202741B20D300D1D4F
:10273000B20E300E182018071226B6B219D22C206D
:10274000280B12254A206726206623D22C30592BCD
:10275000D2772068197553601226B6D22C12190947
:10276000B40B1575F00812046BD5F0FAD267122677
:10277000B67556FA125F61221225E1E55360EF1239
:102780006002302C05C22C122670C28EC2ABD2AFB2
:1027900020B705306AFA808812240C30B706306AF8
:1027A000FA02272079081226C13062DE208FDB2052
:1027B000B7FAD9F27894790B7B007A057C00C26174
:1027C0001226C1208FC420B70520620580F5206243
:1027D000F2A2625002B261EC33FCDAE4D92E20E0BE
:1027E000C303540F6B600280A17894790A75F000DE
:1027F000E6540FF6700205F008D9F5E5F024F8501C
:10280000028087D266D218D27702276E3061082004
:10281000E00302278A808D03540FF6086BFB809A31
:10282000853957755800B23AE5396002D23AA23A72
:10283000B3920AD270223027012278A0760A087655
:1028400003800778A0760A0876010875F06484F69C
:1028500008E5F075F00A84F608A6F0754305D2275E
:10286000227518C0751900751A0112178F2275523A
:1028700000C25D7518C0751900751A0212178F22F3
:10288000D25B7554B475185075190F751AFF12176D
:102890008F22C215122820204D0C75181075190FA3
:1028A000751AFF12178F22204D0C75182075190FFD
:1028B000751AFF12178F2275186075190F751AFF98
:1028C00012178F2275187075190F751AFF12178F4E
:1028D00022C0E0EAC0E0C083C082900242126ACA0D
:1028E000D082D083D0E0AAE0D0E01262697518C02F
:1028F000751900751A0E12178F22302803C380062F
:10290000A290302E01B37836E233F2B4FF02800693
:10291000022A63022B0F2031032037F7D2373013FE
:102920001CC0E0786DE26013C3335005D0E0022B89
:102930000F1204B750F6D0E002293DD0E0E53B602D
:10294000D2B40126D216122861303A15204B0C75EC
:102950005802755702304F03755701853A52022BC2
:102960000F204903122880022B0FB40215303E03BA
:10297000205809207206122892022B011228A70261
:102980002B0FB40308C2581228B7022B0FB4090C3E
:10299000205803204A03022A4B022B0FB40A027468
:1029A0003DB43212122F177518C0751902855C1AC2
:1029B00012178F022B01B4330B122EFD5003122875
:1029C00043022B0FB434087400122836022B0FB4C4
:1029D00035087410122836022B0FB4360874111201
:1029E0002836022B0FB437087420122836022B0F1A
:1029F000B4381B7401F9747CF875300075318C752E
:102A000032F11206DA787CE6122836022B0FB4393E
:102A10001B7401F9747CF875300075318C7532F1D6
:102A20001206DA787CE6122843022B0FB43C061219
:102A300028D1022B01B43D13205808D2581228C4C3
:102A4000022B01C2581228B7022B01751890751974
:102A500009F51A12178F022B0FE53BB40B03A237AF
:102A600022C32270F12031033037EBC23730131C00
:102A7000C0E0786DE26013C3335005D0E0022B0F45
:102A80001204B750F6D0E0022A8CD0E0E53B602279
:102A9000B40107C21612286E8075B402028070B4A9
:102AA0000307D2581228C48066B40908205844305D
:102AB0004A41805BB40A02743DB432028051B4339F
:102AC00002804CB43403022B0FB43503022B0FB435
:102AD0003603022B0FB43703022B0FB43803022B3B
:102AE0000FB43903022B0FB43C03022B0FB43D0388
:102AF000022B0F7518A0751909F51A12178F022BE2
:102B00000F100F03022B0F1261D112053ED20FC21C
:102B100031302803C38006A291302F01B37837E209
:102B200033F2B4FF028006022C7A022D26203203F3
:102B30002038F7D23830131CC0E0786EE26013C33F
:102B4000335005D0E0022D261204B750F6D0E00233
:102B50002B54D0E0E53C60D2B40126D21612286195
:102B6000303A15204B0C755802755702304F0375DB
:102B70005701853A52022D26204903122880022D42
:102B800026B40215303E03205809207206122892FE
:102B9000022D181228A7022D26B40308C2581228A5
:102BA000B7022D26B4090C205803204A03022C62D8
:102BB000022D26B40A02743DB43212122F17751872
:102BC000C0751902855C1A12178F022D18B4330BC9
:102BD000122EFD5003122843022D26B4340874002F
:102BE000122836022D26B435087410122836022D0C
:102BF00026B436087411122836022D26B43708740C
:102C000020122836022D26B4381B7401F9747CF882
:102C100075300075318C7532F51206DA787CE61263
:102C20002836022D26B4391B7401F9747CF87530EE
:102C30000075318C7532F51206DA787CE61228437D
:102C4000022D26B43C061228D1022D18B43D1320C3
:102C50005808D2581228C4022D18C2581228B70298
:102C60002D1875189075190AF51A12178F022D264E
:102C7000E53CB40B03A23822C32270F120320330AA
:102C800038EBC23830131CC0E0786EE26013C333F7
:102C90005005D0E0022D261204B750F6D0E0022CE9
:102CA000A3D0E0E53C6022B40107C21612286E8072
:102CB00075B402028070B40307D2581228C480662B
:102CC000B40908205844304A41805BB40A02743D7C
:102CD000B432028051B43302804CB43403022D2646
:102CE000B43503022D26B43603022D26B437030271
:102CF0002D26B43803022D26B43903022D26B43C08
:102D000003022D26B43D03022D267518A075190A5D
:102D1000F51A12178F022D26100F03022D261261AD
:102D2000D112053ED20FC232302803C38006A292D0
:102D3000303001B37838E233F2B4FF028006022E5D
:102D400045022ED82033032039F7D23930131CC066
:102D5000E0786FE26013C3335005D0E0022ED81242
:102D600004B750F6D0E0022D6BD0E0E53D60D2B460
:102D7000090C205803204A03022E2D022ED8B40A33
:102D800002743DB43212122F177518C075190285DE
:102D90005C1A12178F022ECAB4330B122EFD500389
:102DA000122843022ED8B434087400122836022E9A
:102DB000D8B435087410122836022ED8B4360874E8
:102DC00011122836022ED8B4370874201228360281
:102DD0002ED8B4381B7401F9747CF8753000753145
:102DE0008C7532F71206DA787CE6122836022ED875
:102DF000B4391B7401F9747CF875300075318C7529
:102E000032F71206DA787CE6122843022ED8B43C58
:102E1000061228D1022ECAB43D13205808D25812E7
:102E200028C4022ECAC2581228B7022ECA7518909A
:102E300075190CF51A12178F022ED8E53DB40B0345
:102E4000A23922C32270F12033033039EBC239306A
:102E5000131CC0E0786FE26013C3335005D0E0026A
:102E60002ED81204B750F6D0E0022E6ED0E0E53D29
:102E70006009B40908205844304A41805BB40A0212
:102E8000743DB432028051B43302804CB434030236
:102E90002ED8B43503022ED8B43603022ED8B43758
:102EA00003022ED8B43803022ED8B43903022ED828
:102EB000B43C03022ED8B43D03022ED87518A07579
:102EC000190CF51A12178F022ED8100F03022ED8E4
:102ED0001261D112053ED20FC23320600122C260BE
:102EE000751840751900751A0012178F22E53B649A
:102EF000036008E53C64036002C322D3221205810B
:102F000030130C125847400390FFF112588C22C026
:102F10005C122F2DD05C22301313125847400390BF
:102F2000FFF112588C5005F55C1258E322E55C70F5
:102F300005755C108023B41005755C11801BB411FD
:102F400005755C208013B42005755CFF800BB4FF11
:102F500005755C008003755CFF125AD0E55C22C2E7
:102F60005875186075190F751AFA12178F22D258F2
:102F700075187075190F751AFA12178F22C25875C5
:102F8000186075190F751AE012178F22D25875182C
:102F90007075190F751AE012178F221230821231D4
:102FA000122212308F12311F22B21730131CC0E0D0
:102FB0007871E26013C3335005D0E002300512048B
:102FC000B750F6D0E0022FCAD0E0E53F604524F8C4
:102FD0004005E53F02301EE53FB40904A2148036E7
:102FE000B40A04A216802FB40C03D38029B40D0BAD
:102FF00030350302309CD235D3801BB40E04A215A9
:10300000801402309CB40D0620350302309CC2357A
:10301000C38003A258B3923BB3920B02309C30178B
:103020005E535A03785AA2E2825B4030A2E0825C8F
:103030004012A2E1825D4018C23BA23BB3920B76E4
:103040000002309CB60102801D7601755940801641
:10305000B60202801176027559A0800AB60302807A
:103060000576037559CCE55923F55920E00AC23B92
:10307000A23BB3920B02309CD23BA23BB3920B0219
:10308000309CE53FB40B07D23BA23BB3920B22E549
:103090003FB40B07C23BA23BB3920B2230131CC0C0
:1030A000E07872E26013C3335005D0E00230F612CC
:1030B00004B750F6D0E00230BBD0E0E540604524D4
:1030C000F84005E54002310FE540B40904A2148040
:1030D00036B40A04A216802FB40C03D38029B40D91
:1030E0000B30360302312CD236D3801BB40E04A22F
:1030F00015801402312CB40D0620360302312CC287
:1031000036C38003A258B3923CB3920C02312C0216
:10311000312CE540B40B07D23CA23CB3920C22E523
:1031200040B40B07C23CA23CB3920C2222C0F07503
:10313000F0FAD5F0FD75F064D5F0FDD0F022123133
:103140002D12312D12312D12312D12312D12312D22
:1031500022756A08A2E7B39293C2B412312DC293CA
:10316000D2B412312DC0E0E430B301040030B30119
:10317000040030B30104D36003D5E001C3D0E033D1
:10318000D56AD122D2B4C293D2B312312DC2B412B5
:10319000313ED2B412313E20510620280330772A26
:1031A000788C7601087480F608A20692E430510209
:1031B00074B3F674800830510274B0F608305102CE
:1031C0007480F608F608F602320B788C76030876DF
:1031D00080087480A26B92E5A20692E420280B205E
:1031E0007708A26E92E1A23A92E0F6087480202855
:1031F0001120770EE55B54074480A26D92E5A2088A
:1032000092E4F6087480F608F608F675F007788CF4
:103210007E007F00E62EFEE6123151F62FFF08D524
:10322000F0F2EED333123151F8EFD33368704678B1
:103230008CB6FF417892E644F3046039056CE56C86
:1032400024FE501A756C02202A14D22AE8C0E075B8
:1032500018C0751900751A0312178FD0E0F878920C
:10326000E6205166202863207760788D20E32E20A9
:10327000E21E0232CAE56C6014D56C11302A0EC20F
:103280002A7518C0751900751A0412178F0232CAF0
:10329000788D864308D26779A07A048008788DD229
:1032A0006679947A05D27675F00FE6C4540FF75517
:1032B000F0F5F009E6540FF755F0F5F00908DAEAF1
:1032C000E5F0B40F051977EEC266D2B4C29375F07B
:1032D0000512048320B30612048330B303D5F0F142
:1032E0002220510C75F00312046BD5F0FA123184D0
:1032F0002220510F30760C7518B0751900751A0020
:1033000012178F227005756F1E8002D22222C2987A
:10331000C299322028F8309918C299206505753570
:1033200000800EC0E0C0D075D0101235E9D0D0D0EA
:10333000E020980132C2982065FAC0D0C0E0E8C011
:10334000E0306405C264754900E55024FE40037511
:103350005002E54920E712E54954072324FAC0E06A
:1033600074003434C0E0E59922543F232324EDC097
:10337000E074003433C0E0E59922156E0234EC02AB
:1033800034ECD56EFAB54F08D21A7549000234F202
:1033900002350AB462FA0234EC0234ECB42AF102C7
:1033A00034ECF56E24C6E56E40E624F5E56E50E09B
:1033B000056E0234EC7820F2156E0234EC7821F2BE
:1033C000156E0234EC7822F2156E0234EC7823F29A
:1033D000156E0234EC7824F2156E0234EC7825F286
:1033E000156E0234EC7826F2156E0234EC023520AC
:1033F00000023393000233990002339C000233A28F
:103400000002337A0002337A0002337A0002337A00
:10341000000233B5000233BD000233C5000233CDD4
:10342000000233D5000233DD000233E500023382AF
:1034300000023382000233820002338200023382B0
:1034400000023382000233820002338200023382A0
:103450000002338200023382000233820002338290
:103460000002338200023382000233820002338280
:103470000002338200023382000233820002338270
:103480000002338200023382000233820002338260
:103490000002338200023382000233820002338250
:1034A0000002338200023382000233820002338240
:1034B0000002338200023382000233820002338230
:1034C0000002338200023382000233820002338220
:1034D0000002338200023382000233820002338210
:1034E0000002338200023382000235200549254F55
:1034F000F54FD0E0F8D0E0D0D032800E802A802D79
:103500008030803280348040803EB40908754F009E
:1035100075490080D7B44208754F0075498080CC4A
:10352000754F0075490080CAB51EDF80BFB51FDA30
:1035300080BAF54A80B6F54B80B2B54FCD755020B4
:1035400012354A75490080AA80D6854A37126531FE
:10355000D265E537B44603024136B44704126547E5
:1035600022B4500D854B3612650CC2ACC265D22612
:1035700022B45311854B36E54B700912650CC2AC71
:10358000C265D21D22B4540D854B3612650CC2ACF7
:10359000C265D21C22B4550D854B3612650CC2ACE7
:1035A000C265D21E22B4560D854B3612650CC2ACD4
:1035B000C265D21F22B4570D854B3612650CC2ACC2
:1035C000C265D22022B4580D854B3612650CC2ACB0
:1035D000C265D2212224BF24E64004854B3622C294
:1035E0006522C5382538C53822E53524F0400EE57A
:1035F00035232408C0E074003436C0E022759906F3
:10360000C265753500D2B6228036803B803D803F52
:1036100080408045804D804F805880568054805235
:10362000804D8057800D8015753503F5991235E270
:10363000053522A836E630002CE20236650236ACAB
:10364000753800740380E4E51E80E0E51F80DC022D
:1036500036F1E53875350F80D21217BD1233048864
:103660003680C8E53680C1E536A25892E080B9754B
:103670003503A8360536E676FF80B0E536C313601D
:103680002714700BA23792E0B392E1440480D61461
:10369000700BA23892E0B392E1440880C81470081D
:1036A000A23992E0440C80BD74FC80B9E5361470F8
:1036B000107408A27192E0A27292E1A23A92E280A2
:1036C000A41470107410A23792E0A23892E1A239CB
:1036D00092E280911470087418A22A92E0808614F5
:1036E000700BA27392E0A27492E1023665E4023696
:1036F00065E537B4410675350402362BB4422AE538
:1037000036600330221B53620F53630FC2AFE56371
:10371000B56206D2AFD3023721056353630FD2AF30
:10372000C3756F1E7442023628B444552013F7E562
:1037300036C3137022B3926F122EED404020413DEC
:1037400030420B205705306F348003206F2FA26F5B
:103750009258925702377D926F14C0E003030354CE
:103760000F243DF8D0E0540704FA7400D333DAFD97
:10377000306F05FAE24A8004F4FAE25AF6E537803F
:10378000A5B44B028003023816E53654F8B408128B
:10379000E5365407603714604314604714605C02D8
:1037A00035FDB4200FE5365407605914605C146091
:1037B0005F0235FDB42813E536A2E09258757B010F
:1037C0005003757B02E5370236280235FD751AF481
:1037D000C272C271755701755801805E751AF3D2B5
:1037E0007280EF751AF2D271C27275570175580165
:1037F000C23AA23AB3920AD270803F751AF1D271DE
:10380000C2728031C273C2748039D273C274803381
:10381000C273D274802DB4430FB53603755103754E
:1038200035077536A802362BB44A20E536701920C4
:103830007216751AF0C21512282075181075190F16
:1038400012178FE5370236280235FDB44506753567
:103850000602362BB4510675350C02362BB44D0ECC
:10386000E536121938E5375002B2E7023726B44C74
:103870000675350E02362BB4460280C9B447028065
:10388000C4B44F08C25BC25CC25D80B9B45908C2FF
:103890000075350D02362BB45A08D20075350D026D
:1038A000362B0235FDE571C27A6002D27AE55CF50D
:1038B0005DC25E206609306703023907023E7A1254
:1038C000056F1222261220B370202073082074176F
:1038D000123F6B501212054812257E30670CE543EB
:1038E0006008121F127003023A3075553CD551140E
:1038F00075183075190085511A12178F755103D23A
:103900005C7554B4023E4C12056FE54360F6B40298
:1039100006125061023E7A20764A20270330434443
:10392000B4012E78A0E6B40A28C05C122F17123E0C
:10393000F44012E543B4010878A0E6B40A0280EB33
:10394000D05C023E0DD0E0E55CF55D12053E023E26
:103950007AB4051078A0B60A0B08B601028008B642
:1039600003028003023A0308E675F00AA4082675EC
:10397000F00AA40826C5F0703B78A1B603392027C9
:1039800009C0F0123EF4D0F0502A85F05C85F05D5D
:1039900012053E20270F7518C0751903855C1A1291
:1039A000178F023E7A7518C0751902855C1A1217B6
:1039B0008F023E7A023E0D202709C0F0123EE0D071
:1039C000F050F185F05C20270E7518C0751906853A
:1039D0005C1A12178F800C7518C0751905855C1A52
:1039E00012178F12593C123F3FC209C26ED208D241
:1039F0006D120548122700A266726750030238B3A1
:103A0000023E7A1221897025207308207422123F09
:103A10006B501D12054812270030661112056F12F7
:103A200022267894797C7A05121E6360030238EAB4
:103A3000755500755103C25DC25C205E02C25BC059
:103A400082C083124012D083D0825006123D97026A
:103A50003E7AC082C0831208CFD083D08250061233
:103A60003D97023E7AE58224CEE58334FF5013125F
:103A70003F59400E122EED5006123D3D023E7A0295
:103A80003C29122C704005122E3B5012123D3D0273
:103A90003BE8123D1E023BE8123CFF023BE820726D
:103AA000F1303E032058F1E5426050E542600923C1
:103AB0001204B74003023AC1023AFB123CE0023B57
:103AC000E83013F73025F43050F1A276305201B3CC
:103AD000502930131BC0E07876E26012C3335004E3
:103AE000D0E080D71204B750F7D0E0023AF0D0E02F
:103AF0001263DD5006123D5B023BE830254912633C
:103B000083A2E09223A2E19224A276305201B392E2
:103B100010B4000530102D8020B4012220101A7539
:103B200018C0751900751A0912178F204C06123D1E
:103B300079023BE8123EBD800E1263008009B40298
:103B4000ED2010DB12632930137930131CC0E078AC
:103B500075E26013C3335005D0E0023BC31204B7D3
:103B600050F6D0E0023B69D0E0207A16A276927936
:103B7000858372858273123EA01205597571020207
:103B80003E7A757100E5836572F5F0E582657345EF
:103B9000F07006123DB5023BE87518C07519007546
:103BA0001A0C12178F30790C7518B0751900751A28
:103BB0000012178F123DF375181085721985731A4C
:103BC00012178FD209C26E123E83A2769215D214BA
:103BD0001228201232F1123DF375181085831985D1
:103BE000821A12178F12053E123F625003023E7A6C
:103BF000122EED40F8C206C26BD208D26DC207C2C7
:103C00006C755B001232E1121F8C122700206606D1
:103C1000206711023E7A7894797C7A05121E6360DF
:103C200008023E4C121F1270F8302524E4A22392A1
:103C3000E0A22492E1B403051263558013B4020597
:103C4000126300800BB4010512632980031262D74E
:103C500030131CC0E07873E26013C3335005D0E02A
:103C6000023E4C1204B750F6D0E0023C6FD0E03078
:103C7000530FE58245836009023C81123CC1023E3C
:103C80007AB2581232F130581A7518708583198536
:103C9000821A12178FD206C26BC208C26DC207C247
:103CA0006C801875186085831985821A12178FC267
:103CB00006C26BC208C26DD207C26C12053E023E3C
:103CC0007A125E89C0E0EAC0E0C083C0829004043A
:103CD000126ACAD082D083D0E0AAE0D0E0023DD1FF
:103CE000125E89C0E0EAC0E0C083C0829003B212D5
:103CF0006ACAD082D083D0E0AAE0D0E0023DD112DF
:103D00005E89C0E0EAC0E0C083C0829003DB126A33
:103D1000CAD082D083D0E0AAE0D0E0023DD1125ECA
:103D200089C0E0EAC0E0C083C082900389126ACAF9
:103D3000D082D083D0E0AAE0D0E0023DD1125E89EB
:103D4000C0E0EAC0E0C083C082900360126ACAD0BB
:103D500082D083D0E0AAE0D0E08076125E89C0E015
:103D6000EAC0E0C083C0829002CE126ACAD082D07C
:103D700083D0E0AAE0D0E08058125E89C0E0EAC0BB
:103D8000E0C083C08290027C126ACAD082D083D005
:103D9000E0AAE0D0E0803A125E89C0E0EAC0E0C06C
:103DA00083C082900257126ACAD082D083D0E0AA20
:103DB000E0D0E0801C125E89C0E0EAC0E0C083C0B1
:103DC000829001F0126ACAD082D083D0E0AAE0D0FB
:103DD000E07571007572FF7573FF122F9B1232F13F
:103DE00075182085831985821A12178F12052B12D8
:103DF0002FA222207616E55C046011146570600C19
:103E00007518C0751901855C1A12178F22125E8908
:103E1000C0E0EAC0E0C083C08290022E126ACAD01D
:103E200082D083D0E0AAE0D0E074001257AAC0E0AC
:103E3000EAC0E0C083C08290023D126ACAD082D03C
:103E400083D0E0AAE0D0E012051A802E125E89C06D
:103E5000E0EAC0E0C083C0829001C6126ACAD08284
:103E6000D083D0E0AAE0D0E0122F9B12051A122FC7
:103E7000A27571007572FF7573FFC267C266E55D5A
:103E8000F55C22125E89C0E0EAC0E0C083C0829087
:103E900001DB126ACAD082D083D0E0AAE0D0E0224F
:103EA000125E89C0E0EAC0E0C083C08290021912AD
:103EB0006ACAD082D083D0E0AAE0D0E022125E8924
:103EC000C0E0EAC0E0C083C0829002A5126ACAD0F6
:103ED00082D083D0E0AAE0D0E075F03212058B22C8
:103EE0007408F9747CF875300175310375329812D5
:103EF00006DA80127408F9747CF8753001753103A4
:103F00007532901206DA7881E60856085604602D5C
:103F1000C0E0EAC0E0C083C0829001A3126ACAD0A8
:103F200082D083D0E0AAE0D0E012054812257E308E
:103F30006709E5436005121F126002C322D322C045
:103F4000E0EAC0E0C083C0829002E3126ACAD08275
:103F5000D083D0E0AAE0D0E022E582249CE583343F
:103F6000FF22E582249CE58334FF22A255E58245A9
:103F7000836010E582249CE58334FF5004A25480C2
:103F800002A25622E5822582F582E5833583F583F8
:103F9000E5822582F582E5833583F583E582240079
:103FA000F582E583345BF5837404F97400F87530A9
:103FB000018583318582321206B5227881E654C0AC
:103FC000F5837882E630E402240A2323543C4583B7
:103FD000F5837881E6C4540375F00AA4F5F0E6543D
:103FE0000F25F0030303F5F053F0E085F08254034E
:103FF0004583F5837880E6C4540375F00AA4F5F090
:10400000E6540F25F04582F58222C39582E5F095AE
:104010008322123F847800E2B4FF030240921269C7
:104020000C123FBB787CA68308A6827800E2F58359
:1040300008E2F58208E2F5F008E212400A502B7817
:1040400000E2F58308E2F582787C86F008E612400B
:104050000A50417802E2F58308E2F582787C86F026
:1040600008E612400A402D0240927800E2F58308EB
:10407000E2F582787C86F008E612400A4016780263
:10408000E2F58308E2F582787C86F008E612400AC1
:104090005002C322D322C5382538C53822E555241D
:1040A000E94008C206C26BC209C26E3098EFC298DE
:1040B000E599124096223099FDC299F599124096E1
:1040C00022D206C26BD209C26EC2B6753800740520
:1040D0001240B6E51E1240B6E51F1240B622120489
:1040E0009B12049B12049B1240C1E5371240B6E5B7
:1040F000381240B63099FD22120C40024101120BD9
:10410000DCC0E01240C1E5371240B6D0E01240B644
:10411000E5381240B63099FD2212049B1240C1E5E9
:10412000371240B6797CE71240B609DDF9E538125E
:1041300040B63099FD22751A00755519D228E53F11
:10414000600B54F87007C23BA23BB3920BE5406092
:104150000B54F87007C23CA23CB3920CD2A0C28EA2
:10416000C28CC2ADC2ABC2ACC2AF7581CD9041783A
:10417000C082C08375D00032D2AFD28CC0E0EAC01A
:10418000E0C083C08290018E126ACAD082D083D0F0
:10419000E0AAE0D0E0C0E0EAC0E0C083C0829000C6
:1041A00069126ACAD082D083D0E0AAE0D0E012655A
:1041B0000CC2ACD2991240DEB20312181875551910
:1041C000D2980241EAB40922F53812409DB51E2763
:1041D00012409DB51F2112409DB4461B12409DAF59
:1041E0003812409D6F70101240DED2B6C206C26B0C
:1041F000C209C26E12409DB40ACBF53812409DB57B
:104200001EF512409DB51FEF12409DF537B46D03AA
:1042100002429AB46E030242B3B46F030242EAB49C
:104220007003024337B4710302434BB47303024378
:104230005CB4740302435EB47503024372B4760344
:1042400002438AB4770302439EB478030243B2B4B4
:1042500079030243D3B47A030243EFB46C030244FC
:1042600003B46B03024425B46A03024460B46903D7
:1042700002447CB468030244BEB467030244D6B46B
:1042800066030244F1B465030245B5B46403024D0C
:10429000D7B46103024E320241EAAF3812409D6F3B
:1042A00070F51240DED2B675F01E12046BD5F0FA2E
:1042B00002669B12409DFD1424E0402B12409D2479
:1042C00000FC7B0012409DFEAF3812409D6F7017BE
:1042D0008EF0EDF9747CF88B308C3185F03212065B
:1042E000DA1241197555190241EA12409DFD145424
:1042F000E070F412409D2400FC247140EA7B02121D
:10430000409DFEEDFA787C12409DF608DAF9AF3850
:1043100012409D6F70D1D206C26BD209C26E8EF070
:10432000EDF9747CF88B308C3185F03212062F1247
:1043300040E775551980B0AF3812409D6F70A812D4
:1043400009E61240DE7555190241EAAF3812409D68
:104350006F70091240FE7555190241EA80891240BA
:104360009DFD1424E0404812409D2400FC7B010286
:1043700042C412409DFD1454E0703412409D24004C
:10438000FC2425402A7B030242FFAF3812409D6F78
:10439000701D0243AF1240E77555190241EAAF386C
:1043A00012409D6F70091240F87555190241EA02DA
:1043B00042E779207D0712409DF309DDFCAF3812FA
:1043C000409D6F70EA1257C640E51268ED1240E753
:1043D0000241EAAF3812409D6F70D412690C12048A
:1043E0009B1240C1E5371240B612158B0241EAAF6D
:1043F0003812409D6F70661211AD1240DE7555196E
:104400000241EA12409DFE12409DFD12409DFCAF0C
:104410003812409D6F704612094C40411240DE75C3
:1044200055190241EA12409DFE12409DFDAF38121F
:10443000409D6F702812091D12049B12049B1240AC
:10444000C1E5371240B6EE1240B6ED1240B6EC129E
:1044500040B6E5381240B63099FD0241EA0242E723
:10446000AF3812409D6F70F512049B12049B1240EE
:10447000C1E5371240B612161B0241EAAF381240AE
:104480009D6F70D9120BD460027401C0E0120C3819
:1044900060027402D0F045F0700A120A31121ACA92
:1044A0001211ADE4C0E01240C1E5371240B6D0E0D1
:1044B0001240B6E5381240B63099FD0241EA12408A
:1044C0009DFD1454E0702712409D2400FC2471408F
:1044D0001D7B000242FF12409DFD1454E0700F123C
:1044E000409D2400FC242540057B010242FF02423E
:1044F000E7AF3812409D6F70F512049B12049B12B7
:1045000040C1E5371240B674011240B6744C1240F7
:10451000B6746A1240B674461240B674351240B68C
:1045200074001240B6748D1240B674201240B674F6
:10453000DA1240B674001240B6740F1240B674A07E
:104540001240B674801240B674001240B674001265
:1045500040B674201240B674001240B67400124087
:10456000B674001240B674001240B674001240B621
:1045700074001240B674001240B674001240B67453
:10458000001240B674001240B674001240B67400B7
:104590001240B674001240B674001240B674001295
:1045A00040B674001240B6E5381240B63099FD02AC
:1045B00041EA0242E712409DF58312409DF58224B4
:1045C00060E58334F040EB12484912409DFD1454DD
:1045D000E070DF780012409DF208DDF9AF3812403C
:1045E0009D6F70CE1240DE75F00512046BD5F0FAA7
:1045F0001240E7751A013013B93012B61249BC12D5
:1046000049A2124857121F8C789479007A0A75F0E3
:104610000FE3540FF652F00809DAF643F0F0E5F034
:10462000047894797C7A05121E63600B1246CD5093
:1046300006751A040245B21249A2124857121F8C7D
:1046400078A0790A7A0675F00FE3540FF652F00855
:1046500009DAF643F0F0E5F00478A079817A0312E4
:104660001E63600B12476B5006751A060245B212A4
:1046700049A2124A05751A650241EAC0E07830E5A0
:1046800083F208E582F2D0E022C0E07832E583F2DE
:1046900008E582F2D0E022C0E07830E2F58308E25B
:1046A000F582D0E022C0E07832E2F58308E2F582BC
:1046B000D0E022E5822400F582E583341BF58322D5
:1046C000E5822400F582E583343BF58322124857C6
:1046D000AB83AC82901B00C0837900753003858367
:1046E000317532009000361205E11207581205E1CB
:1046F0001207D49000367A80E0A3F5F0E0A36C7046
:1047000005E5F06B6017DAF0D0830583740024C0F0
:10471000E58334C550C1740512481AD322D083EA08
:104720002AF5F0E4C395F0F58212467B789479007F
:104730007A0A75F00FE3540FF652F00809DAF643DF
:10474000F0F0E5F004600C1220B8700A740612480C
:104750001AD3221220B8E5822582F582E5833583BB
:10476000F5831246B3124689024BDC124857AB83DD
:10477000AC82903B00C0837900753003858331752E
:1047800032009000361205E11207581205E11207B7
:10479000D49000367A80E0A3F5F0E0A36C7005E5D4
:1047A000F06B6017DAF0D0830583740024C0E583D2
:1047B00034A550C1740512481AD322D083EA2AF5D1
:1047C000F0E4C395F0F58212467B78A0790A7A0668
:1047D00075F00FE3540FF652F00809DAF643F0F0E3
:1047E000E5F004601D122199701BAB83AC82124866
:1047F00057EBB58306ECB58202C322740412481A43
:10480000D322122199E5822582F582E5833583F54D
:10481000831246C0124689024BDCF51A22C082C0C0
:1048200083E5831257AAD083D082C082C083E582F9
:104830001257AAC083C082C0E07420126A6ED0E012
:10484000D082D083D083D08222C0E07834E583F256
:1048500008E582F2D0E022C0E07834E2F58308E295
:10486000F582D0E022C083C082C0E074D3126A6EA9
:10487000D0E0D082D083C083C082C0E0746F126A5F
:104880006ED0E0D082D083C083C082C0E0743A1280
:104890006A6ED0E0D082D0837881E61257AA7882FF
:1048A000E61257AA7883E61257AAC083C082C0E0F6
:1048B0007420126A6ED0E0D082D083C083C082C0E0
:1048C000E07420126A6ED0E0D082D083C083C082B0
:1048D000C0E07420126A6ED0E0D082D083C083C062
:1048E00082C0E07420126A6ED0E0D082D083C08390
:1048F000C082C0E074D2126A6ED0E0D082D083C091
:1049000083C082C0E0746E126A6ED0E0D082D08321
:10491000C083C082C0E0743A126A6ED0E0D082D008
:104920008378A0E61257AA78A1E61257AA78A2E6E1
:104930001257AA78A3E61257AA78A4E61257AA78C3
:10494000A5E61257AA120CD222C083C082C0E0741E
:10495000D2126A6ED0E0D082D083C083C082C0E021
:10496000742E126A6ED0E0D082D083C083C082C021
:10497000E0746B126A6ED0E0D082D083C083C082B4
:10498000C0E0746F126A6ED0E0D082D083C083C062
:1049900082C0E0746E126A6ED0E0D082D083120CB6
:1049A000D22274001240B674001240B67400124055
:1049B000B674001240B674001240B62275831B759F
:1049C000821B75F040C0F0C082C0837530018583C2
:1049D000317532001205E1120758D083D082C082AF
:1049E000C0837530038582317532001205E11208EB
:1049F0005AD083D08205830582D0F0D5F0C77533B5
:104A0000FF7534FF227401F97418F87530007531A0
:104A1000007532001206DA7401F97419F875300164
:104A20007531D97532FF1206DAAC18124857E58293
:104A30002420F582E583347DF583C082C083740130
:104A4000F97442F87530008583318582321206DAB6
:104A5000D083D0827401F97410F8753000858331E9
:104A60008582321205FE7810E2F5F0E5182542C382
:104A700095F0F518124857E58275F008A42420F542
:104A800082500205F0A8F0E58375F008A428240000
:104A9000F5837408F9747CF875300085833185825C
:104AA000321206DA787CE5187A082608DAFCF5185E
:104AB000789479007A0A75F00FE3540FF652F008F3
:104AC00009DAF643F0F0E5F00412567378A0790A9B
:104AD0007A0675F00FE3540FF652F00809DAF64340
:104AE000F0F0E5F00412567B7408F9747CF8753028
:104AF0000085833185823212062F787CE5187A088A
:104B0000C39608DAFBF518124857C3E58233F582DD
:104B1000E58333F583C3E58233F582E58333F5839B
:104B2000E5822400F582E583245BF583C082C0839F
:104B30007404F9747CF875300185833185823212F2
:104B400006DAD083D0827404F97412F875300185C6
:104B500083318582321205FE787C7912E5197A0458
:104B600026F5F0E3C5F0C395F00809DAF3F51974FA
:104B700001F97418F87530007531007532001206AD
:104B80002F7401F97419F87530017531D97532FF38
:104B900012062F75831B75821B75F040C0F0C08212
:104BA000C0837530038583317532001205E1120729
:104BB00058D083D082C082C0837530018582317520
:104BC00032001205E112085AD083D0820583058293
:104BD000D0F0D5F0C77533FF7534FF221246A5E536
:104BE000828583F0124697C39582C0E0E5F09583F5
:104BF000D0F045F07002C3225003024CF71246A5D4
:104C0000C0E0C3E58224FEF582E58334FFF583D05E
:104C1000E0124689E5828583F0124697B58207E562
:104C2000F0B58302C322124697AF831246A5EFB5B3
:104C30008310AE82900034787CE0F6A308E0F602A0
:104C40004C5A7EFE8F8305837402F9747CF87530AC
:104C5000038583317532001206DA79007530038FCF
:104C6000317532009000361205E11207581205E145
:104C70001207D48F837582001246977D00E5836FFB
:104C80007002AD82ED2436F58275830050020583F3
:104C9000C3EE9D20E05A03FCC082C083A3A3E0FAC8
:104CA000A3E0FBD083D082EAF0A3EBF0A3DCE9EE33
:104CB0002436F58275830050020583787CE6F0A3E4
:104CC00008E6F079007530038F31753200900036B8
:104CD0001205E11208401205E112085A85303385A9
:104CE00031341246A5EFB58303024DCB0F024C2B96
:104CF000740812481AD322124697AF831246A5EFC2
:104D0000B58310AE82900034787CE0F6A308E0F61C
:104D1000024D2B7E008F8315837402F9747CF87525
:104D200030038583317532FE1206DA79007530035F
:104D30008F317532009000361205E11207581205C6
:104D4000E11207D41246977DFEE5836F7002AD82B3
:104D5000ED2436F58275830050020583C3ED9E2055
:104D6000E06B03FCC0E0C3E58224FEF582E58334FA
:104D7000FFF583D0E0C082C083E0FAA3E0FBA3EAA2
:104D8000F0A3EBF0D083D082DCDAEE2436F5827526
:104D9000830050020583787CE6F0A308E6F07900F2
:104DA0007530038F317532009000361205E112081C
:104DB000401205E112085A8530338531341246A578
:104DC000EFB58303024DCB1F024CFCC322740912C2
:104DD000481AD3220242E712409DF58312409DF506
:104DE00082AF3812409D6F70EBC01EC01F85831EBE
:104DF00085821F121DE87401F9747CF87530007506
:104E000031007532001206DA787CE6C3951EC39530
:104E10001FD01FD01E251E251FF67401F9747CF8C3
:104E200075300075310075320012062F1240DE0217
:104E300041EA12409DF583AF3812409D6F70951284
:104E4000049B12049B12049B1240C1E5371240B62A
:104E500074001240B6E51A1240B674001240B674DF
:104E6000001240B674001240B674001240B6E53825
:104E70001240B63099FD0241EA904E81C082C08353
:104E8000327581CD75D00002669BC082C083E582F9
:104E90002420F582E583347DF5837401F97442F8AA
:104EA00075300085833185823212062FD083D082FF
:104EB000C082C083E58275F008A42420F5825002E8
:104EC00005F0A8F0E58375F008A4282400F58374A4
:104ED00004F9747CF87530008583318582321206BE
:104EE0002FA3A3A3A3747C2404F5F07404F9E5F0C4
:104EF000F875300085833185823212062FD083D039
:104F000082C21222120BDCC0E07401F9747CF875C5
:104F100030007531007532001206DA787CE6D0F088
:104F2000C395F0F67401F9747CF8753000753100A2
:104F300075320012062F2212051AC2AF80FE3013FE
:104F40001CC0E07873E26013C3335005D0E0024F19
:104F5000EE1204B750F6D0E0024F5DD0E0C0E0EAB8
:104F6000C0E0C083C082900456126ACAD082D08347
:104F7000D0E0AAE0D0E0C206C26BD208D26DC20770
:104F8000C26C120548122700206606206730024FC7
:104F9000EE1205811220B37055123F62405020730B
:104FA0000820744C123F6B504712054812257E3082
:104FB000673CE5436038121F127033024FF0E5433F
:104FC000602C1205811221897024123F62401F203B
:104FD000730820741B123F6B5016120548122700ED
:104FE00030660B7894797C7A05121E636002D322B6
:104FF000305331E5824583602BE54260092312047A
:10500000B74003025009025024C0E0EAC0E0C08368
:10501000C082900404126ACAD082D083D0E0AAE091
:10502000D0E080CAB258C31232F130581A751870E5
:1050300085831985821A12178FD206C26BC208C2E5
:105040006DC207C26C801875186085831985821A35
:1050500012178FC206C26BC208C26DD207C26CC3E0
:105060002278A0E6B40A1708E6B4055E122EED40D9
:1050700009124F3E400412053E2212051A2275F015
:105080000AA4F5F008E625F0B4633FC206C26BD26D
:1050900009D26ED208D26DC207C26CC0E0C0E0EA8D
:1050A000C0E0C083C08290013A126ACAD082D08325
:1050B000D0E0AAE0D0E012054812270090000012CC
:1050C0001F8C20660920672BD0E012051A221205DA
:1050D000817894797C7A05121E6370EC30553A120F
:1050E000054812257E3067E0120581121F1270D824
:1050F000025119120581E54360CE121F1270C930AA
:1051000055171205481227003066BD1205817894A4
:10511000797C7A05121E6370AF120548C0E0EAC0C0
:10512000E0C083C0829002F8126ACAD082D083D0D5
:10513000E0AAE0D0E0D0E0B40B081254E4405602FC
:105140005359B40C08125525404B025359B40D085D
:105150001255504040025359B40E3D12555F401C49
:10516000C0E0EAC0E0C083C08290033C126ACAD0AB
:1051700082D083D0E0AAE0D0E0025368C0E0EAC069
:10518000E0C083C08290034E126ACAD082D083D01E
:10519000E0AAE0D0E0025355B40F5212690CC0E00F
:1051A000EAC0E0C083C08290014C126ACAD082D0AB
:1051B00083D0E0AAE0D0E01256D1402EF824DC40A3
:1051C00029E87880F6C083C082C0E0743A126A6E23
:1051D000D0E0D082D0831256D1400FF824A0400AEC
:1051E000E8787FF61268ED025359025355B4100265
:1051F00080030252D212690CC0E0EAC0E0C083C052
:105200008290015F126ACAD082D083D0E0AAE0D037
:10521000E012257A20590612257A3059CD12190943
:10522000C0E0C083C082C0E02410126A6ED0E0D01B
:1052300082D083D0E0F824F640B0E8131354C0784D
:1052400081F6C083C082C0E0742F126A6ED0E0D0B5
:1052500082D0831256D140926090F824ED408BE8C2
:105260007882F6C083C082C0E0742F126A6ED0E0EC
:10527000D082D0831256D140566054F824CE404F8D
:10528000E8788146F6C083C082C0E0742F126A6E4F
:10529000D0E0D082D08312257A20590612257A30A8
:1052A000592D121909C0E0C083C082C0E024101239
:1052B0006A6ED0E0D082D083D0E0F824F94010E8C4
:1052C00013131354C0788246F61268ED0253590244
:1052D0005355B41115121921B4010C121921B40738
:1052E0000612556E025359025355B41339203DF737
:1052F0001227002067243066EE121F347057C0E07A
:10530000EAC0E0C083C082900316126ACAD082D07D
:1053100083D0E0AAE0D0E0024F37E5436037121FA8
:10532000507032024F37B4632C702A121921F5786D
:1053300090011F700390012CC0E0EAC0E0126ACA1D
:10534000D0E0AAE0D0E075F06412046BD5F0FA0268
:10535000535902535512051A22124F047518C0757D
:105360001900751A0A12178F12053E22754200782D
:105370007C75F00876FF08D5F0FA22EFC0E0C25F36
:10538000789979817A06EA30E004E6088002E6C47A
:10539000540FFFEA30E004E7098002E7C4540FB479
:1053A0000F10BF0F10EA6406600B205F1ED0E0FFF5
:1053B000E422BF0F06D0E0FF740122205FF7F5F072
:1053C0008F486F6002D25FDABD80DFE5F0C3954899
:1053D0005002F4041460D6B408DB80D17894797C50
:1053E0007A057401B6FF02800FB7FF02800AE667F4
:1053F00070060809DAF8E422740122125406E582E4
:1054000045837001D3228005D0E002545712192140
:10541000C0E024F640F2D0E075F00AA4F5828005E1
:10542000D0E0025457121921C0E024F640F2D0E037
:10543000258275F00AA4F58285F0838005D0E0020C
:105440005457121921C0E024F640F2D0E02582F52D
:105450008250020583C322D322C082C08390000001
:10546000121FE81253DC701AE5828583F0D083D0D6
:1054700082B5821FC5F0B5831AC082C083F58385CB
:10548000F082A3E583B40FD8E582B4A0D3D083D053
:1054900082C322D322C082C083900000121FE81270
:1054A000537B701AE5828583F0D083D082B5821F4A
:1054B000C5F0B5831AC082C083F58385F082A3E569
:1054C00083B40FD8E582B4A0D3D083D082C322D3D3
:1054D00022122700306631125673121F66C32290C3
:1054E000000080081253FB401F12054812270030AD
:1054F0006616120581121F8C1256731254594008F9
:10550000754200124E8AC322D32212257E3067F8DC
:10551000E54324FD24FC40F012567B121F79C32280
:1055200090000080081253FB40DE12054812257ED1
:105530003067D5121F8C12567BE543600B24FD2487
:10554000FC40C512549540C0754200124E8AC322D9
:105550001253FB400812536C124E8AC322D32212FC
:1055600053FB4008121F8C1255BDB322D322C21226
:1055700090002874D8F974FFF8753001858331855F
:105580008232120B8675830175F01E75300085839B
:1055900031753200C0F0C0831205E1120B5AD0837E
:1055A0000583D0F0D5F0E4907D007420F974FFF805
:1055B000753001858331858232120B8622787CE634
:1055C000080808080856B4FF02D322C322751E300B
:1055D000751F30C276C27775F005C0F0C206C26B87
:1055E000D209D26EC208C26DC207C26C12536C12CD
:1055F0002700D0F0206609206706D5F0DD0256446A
:10560000125693403F12053E7881E6B4FF05C3224F
:1056100075F005C0F0122700D0F0206706D5F0F332
:10562000025644E543B4021C78A0E624F64015086F
:10563000E624F6400F78A0E62430F51E08E6243074
:10564000F51FC32212051AD3227547008003754740
:1056500001C25A12270020670B30660A0547E5474A
:1056600024F550EFD322E5476007D25AB40A0274FA
:1056700000C3227894797C7A05800678A079817AB3
:1056800003E608540FC4F5F0E608540F45F0F70997
:10569000DAEF22206631306736E543600624FD24C8
:1056A000FC402C12567B12054875F005C0F01226FE
:1056B000FCD0F0206611205906D5F0F00256CF122A
:1056C0001909B40B0A8003125673754200C322D322
:1056D0002212257A20590612257A30594D121909BD
:1056E000C0E0C083C082C0E02410126A6ED0E0D057
:1056F00082D083D0E0F824F6403012257A20590673
:1057000012257A305924121909C0E0C083C082C022
:10571000E02410126A6ED0E0D082D083D0E0F5F0A1
:1057200024F64006E8C445F0C322D32212573C7544
:10573000F06412046BD5F0FA1204ED2275F03C12FD
:10574000058BC2A075F03C12058BD2A075F0141227
:10575000058BC2A075F03C12058BD2A075F0141217
:10576000058BC2A075F01412058BD2A075F014122F
:10577000058BC2A075F01412058BD2A02275F00A19
:1057800084C0F0C083C082C0E02410126A6ED0E0F2
:10579000D082D083D0F0C083C082C0E0E5F0241076
:1057A000126A6ED0E0D082D08322C083C082C0E073
:1057B000C4540F2410126A6ED0E0540F2410126AE1
:1057C0006ED082D083227825E254C07078E275F0E2
:1057D0000A84C445F0787EF67824E254C07066E20C
:1057E00075F00A84C445F0787FF67823E254E070BF
:1057F00054E275F00A84C445F07880F67822E260BD
:105800004454E07040E275F00A84C445F0C0E0788A
:1058100020E2030354C0D0F045F07881F67821E20D
:10582000602354F0701FE275F00A84C445F0C0E0B4
:105830007826E254F8700EE2C42354E0D0F045F02C
:105840007882F6C322D32290000075F019C0F0745C
:1058500002F9747CF8753001858331858232120635
:10586000DA787DB6FF02800E18E55C301305B4FFD0
:1058700002E570666011E5822410F582500205830E
:10588000D0F0D5F0C8C322D0F0A3D32230134DE519
:105890008224FFF582E58334FFF58375F019E582F4
:1058A0002480E58334FE5005900000800AE58224C0
:1058B00010F58250020583C0F07402F9747CF8750B
:1058C00030018583318582321206DA787DB6FF0297
:1058D000800518E6B55C07D0F0D5F0C2C322D0F041
:1058E000A3D322C0E0EAC0E0C083C082900172125C
:1058F0006ACAD082D083D0E0AAE0D0E07408F974FC
:105900007CF87530018583318582321206DA787C25
:105910007A08126B15E5822408F58250020583741B
:1059200008F9747CF875300185833185823212065E
:10593000DA787C7A07126B15220259C4C083C082C0
:10594000C0E074D1126A6ED0E0D082D083301AE900
:10595000C21A1257C640E21268EDC0E0EAC0E0C0C9
:1059600083C082900087126ACAD082D083D0E0AA16
:10597000E0D0E00259E07822E212577DC083C08275
:10598000C0E0742F126A6ED0E0D082D0837821E21A
:1059900012577DC083C082C0E07420126A6ED0E0CE
:1059A000D082D0837823E212577DC083C082C0E0CA
:1059B000743A126A6ED0E0D082D0837824E2125713
:1059C0007D025ABFC0E0EAC0E0C083C08290008D73
:1059D000126ACAD082D083D0E0AAE0D0E012690C6B
:1059E0007881E6C45403C083C082C0E02410126AE8
:1059F0006ED0E0D082D083E6540FC083C082C0E076
:105A00002410126A6ED0E0D082D083C083C082C0DE
:105A1000E0742F126A6ED0E0D082D0837882E6C420
:105A20005401C083C082C0E02410126A6ED0E0D05E
:105A300082D083E6540FC083C082C0E02410126A73
:105A40006ED0E0D082D083C083C082C0E0742012C8
:105A50006A6ED0E0D082D0837880E6C4540FC083D1
:105A6000C082C0E02410126A6ED0E0D082D083E6FB
:105A7000540FC083C082C0E02410126A6ED0E0D000
:105A800082D083C083C082C0E0743A126A6ED0E0D4
:105A9000D082D083787FE6C4540FC083C082C0E038
:105AA0002410126A6ED0E0D082D083E6540FC083F7
:105AB000C082C0E02410126A6ED0E0D082D0833061
:105AC000130A12584750051258E38003125AD02285
:105AD000C0E0EAC0E0C083C082900172126ACAD0FE
:105AE00082D083D0E0AAE0D0E0E55CB4FF0690026B
:105AF0006C025B39B400069000AC025B39B410064E
:105B00009000B5025B39B411069000BE025B39B457
:105B100020069000C8025B39E55C75F06484C0F033
:105B2000C083C082C0E02410126A6ED0E0D082D060
:105B300083D0E012577D9000F4C0E0EAC0E0126A22
:105B4000CAD0E0AAE0D0E022202501227582051209
:105B50006267604675F00212046BD5F0FAD582EFE9
:105B6000C0E0EAC0E0C083C08290022E126ACAD0B0
:105B700082D083D0E0AAE0D0E074011257AAC0E03E
:105B8000EAC0E0C083C08290023D126ACAD082D0CF
:105B900083D0E0AAE0D0E01262697475783D120506
:105BA0009C502E207B2DD27BC0E0EAC0E0C083C099
:105BB00082900242126ACAD082D083D0E0AAE0D09A
:105BC000E01262697518C0751900751A0D12178FE9
:105BD00022C27B12690C204404204547227880E6CB
:105BE000543FF5F07939E365F0703509E3787F6665
:105BF000702E20462AD246C0E0EAC0E0C083C082B0
:105C0000900242126ACAD082D083D0E0AAE0D0E0EB
:105C10001262697518C0751900751A0D12178F2256
:105C20003045437880E6543FF5F0793BE365F0700A
:105C30003509E3787F66702E20462AD246C0E0EA16
:105C4000C0E0C083C082900242126ACAD082D08370
:105C5000D0E0AAE0D0E01262697518C0751900752D
:105C60001A0D12178F22C24622C2AC1217BD602431
:105C7000F518881912122053620F53630FC2AFE553
:105C800063B56206D2AFD3025C92056353630FD251
:105C9000AFC380D7D2AC227E007F7090000075F039
:105CA00000E49325F0F5F0A3C3E5829EE5839F40D1
:105CB000F0E5F0700122E5F0C0E0C083C082C0E0F2
:105CC00074D2126A6ED0E0D082D083E5831257AAD4
:105CD000E5821257AAC083C082C0E0743A126A6E8D
:105CE000D0E0D082D083C083C082C0E07420126A2A
:105CF0006ED0E0D082D083D0E01257AAC0E0EAC0D4
:105D0000E0C083C0829000FA126ACAD082D083D0E9
:105D1000E0AAE0D0E0C2ADC2ACD22812050520A0B6
:105D2000FA75F0C812046BD5F0FA30A0FD75F0C812
:105D300012046BD5F0FA12650C2275F06412087328
:105D400020E51830E31522120483B203121818124A
:105D50000483B203121818D5F0ED22C2AFB20312B9
:105D60001818120483B203121818120483D5F0CD48
:105D7000C2A075F032125D47D2A075F032125D47B5
:105D8000C2A075F032125D47D2A075F032125D47A5
:105D900075F096125D4780D82230133C7400784D20
:105DA0001205AB40337F087E007478783D12059C65
:105DB000CE13CE05E0DFF420290E7400785D1205C5
:105DC000AB5005EE655E60108E5E8E5C7518C0751A
:105DD0001904855C1A12178F22C2AF751810751935
:105DE0000FF51A12178FD2AF223013097401784DB4
:105DF0001205AB5001227477783D12059CE492E0C5
:105E0000C0E07476783D12059CD0E033FE20290E68
:105E10007401785D1205AB5005EE655F60D78E5F4B
:105E2000EE20E10630E02E025E7230E017A27272C0
:105E30007150C2C272C27175570175580174F8125F
:105E40005DD980B1D272C27175570175580174F76E
:105E5000125DD980A020719DD271C27275570175F3
:105E60005801C23AA23AB3920AD27074F6125DD9BE
:105E70008083A23A827140F8D271C272C215122890
:105E80002074F5125DD9025DF5C082C083C083C065
:105E900082C0E0126983D0E0D082D083C083C08208
:105EA000C0E0EEC0E0EFC0E0126D10D0E0FFD0E047
:105EB000FED0E0D082D083C0E0EEC0E0EFC0E0C012
:105EC00083C082906CF8126D2AD082D083D0E0FF1C
:105ED000D0E0FED0E0C083C082C0E0740C126B8DB5
:105EE000D0E0D082D083C083C082C0E07406126B41
:105EF00075D0E0D082D083126B27D083D08222C0AD
:105F000082C083EAC0E0E8C0E0900190EF75F01035
:105F1000A42582F582E5F03583F5837410F97400C9
:105F2000F87530018583318582321206B57800E23A
:105F3000B4FF03025F548EF0E270027420C0F012CE
:105F40006A6ED0F008D5F0F0D3D0E0F8D0E0FAD007
:105F500083D08222C3D0E0F8D0E0FAD083D082226E
:105F600022C0E0E578B4010620670620666CD0E028
:105F700022C0E0EAC0E0C083C082900099126ACAE1
:105F8000D082D083D0E0AAE0D0E078A0E543602DB5
:105F9000F9E6B40A14C083C082C0E0742A126A6EA3
:105FA000D0E0D082D083025FBAC083C082C0E02438
:105FB00010126A6ED0E0D082D08308D9D4C083C0DA
:105FC00082C0E07423126A6ED0E0D082D08375F074
:105FD000C812046BD5F0FA026083126B27789479AB
:105FE0000AE6C083C082C0E02410126A6ED0E0D0FE
:105FF00082D08308D9EB75F0C812046BD5F0FA0291
:106000006083C0E0E578B4027AC083C082C0E074E7
:10601000D1126A6ED0E0D082D083E4A23E92E0C07A
:1060200083C082C0E02410126A6ED0E0D082D08398
:10603000E4A27292E0C083C082C0E02410126A6EB3
:10604000D0E0D082D083E4A24292E0C083C082C07C
:10605000E02410126A6ED0E0D082D083E4A257927E
:10606000E0C083C082C0E02410126A6ED0E0D0820B
:10607000D083C083C082C0E07420126A6ED0E0D0AA
:1060800082D083D0E022C0E0E578B4022AC083C089
:1060900082C0E074D2126A6ED0E0D082D083EF1258
:1060A00057AAEE1257AAC083C082C0E07420126AB9
:1060B0006ED0E0D082D083D0E022C0E0E578B40496
:1060C000530260CBC0E0E578B40349C083C082C00E
:1060D000E074D2126A6ED0E0D082D0837F08788CD0
:1060E000E688F0C0F01257AAD0F0A8F008DFF175EA
:1060F00056FA3059FA121909B40BF4C0E0EAC0E0BC
:10610000C083C082900099126ACAD082D083D0E046
:10611000AAE0D0E0D0E022C083C082C0E074D112F7
:106120006A6ED0E0D082D083C083C082C0E0744960
:10613000126A6ED0E0D082D083C083C082C0E07487
:1061400044126A6ED0E0D082D083C083C082C0E0A7
:10615000743A126A6ED0E0D082D083E5831257AAD7
:10616000E5821257AAC083C082C0E07420126A6E12
:10617000D0E0D082D08322C2A075F01412046BD577
:10618000F0FAD2A075F01412046BD5F0FA22C2A076
:1061900075F03C12046BD5F0FAD2A075F01412041D
:1061A0006BD5F0FA2212617712617712618E12615B
:1061B0007775F06412046BD5F0FA2212618E1261C9
:1061C0007712617712617775F06412046BD5F0FA7B
:1061D00022305809D206C26BC207C26C22C206C264
:1061E0006BD207C26C2230134930131CC0E07874A4
:1061F000E26013C3335005D0E002621E1204B750B0
:10620000F6D0E0026208D0E0D27320290320752284
:106210007518C0751900751A0F12178F8014C27384
:1062200020290330750C7518C0751900751A1012E5
:10623000178FA273927522120725C20512181874BF
:1062400054120742E41206FF120712F5F0644825C3
:106250006833F568E5F02569B2E003F569D9E9D25C
:1062600005121818222222E4227583DD75F01075BC
:106270003003858331753200C083C0F01205E1120E
:106280000B5AD0F0D0830583D5F0E47533FF753415
:10629000FF126266220262C8C082C083758205C096
:1062A00082126267D082601CC2A075F00F12046B6C
:1062B000D5F0FAD2A075F00512046BD5F0FAD582AC
:1062C000DE126269D083D082E5822400C0E0E583DB
:1062D00034DDF8D0E0C322126298C082C083F58218
:1062E0008883787C76007401F9747CF875300385B6
:1062F000833185823212062FD083D08212626622C9
:10630000126298C082C083F5828883787C7602749A
:1063100001F9747CF8753003858331858232120669
:106320002FD083D08212626622126298126298C0C5
:1063300082C083F5828883787C76017401F9747C4D
:10634000F875300385833185823212062FD083D0D1
:106350008212626622126298C082C083F5828883AC
:10636000787C76037401F9747CF875300385833189
:1063700085823212062FD083D08212626622126288
:10638000958003126298C082C083F582888374016D
:10639000F9747CF87530038583318582321206DA10
:1063A000787CE6B40102800CB402028007B40302D8
:1063B00080027400D083D08222120725C2051218F1
:1063C000187454120742E41206FF120712B40205B1
:1063D0007568018002D9F3D2051218182275680079
:1063E0007583DD75F00F753003858331753200C01C
:1063F00083C0F01205E11207581205E1790012631B
:10640000B9D0F0D0830583E5687028D5F0D8753011
:1064100003858331753200C0E01205E1120758127E
:1064200005E179A01263B97533FF7534FFE5687033
:1064300002D322C322C28C758A45758C5DD28CC072
:10644000D0C0E0C0F075D008D26A202804E55660BC
:1064500005B203121818121855051DE51D20E03568
:1064600020E132202836206E04A23A9209E51D3040
:10647000E203122FA9E51D541F7010E4B55725B58E
:106480005244B55453B56F5BB5555DE4B55645B54B
:106490005364B55065D0F0D0E0D0D032E51D541F24
:1064A00060E680F1304F0CE55824C24003D558CF48
:1064B00075583CD557C9C2142071C4C23AA23AB328
:1064C000920AD27080B9D552B9C2147554B4D25D53
:1064D000D26080AE155680B7D554AAC25BC25CC2EA
:1064E0005D80A2D56FA280A0D555A075510330283C
:1064F00003024E79808F15538098D55098D26480CE
:1065000094C2B6206502D2B612650C3275C800C2BC
:10651000ADC2AC75CBFF75CA9875CDFF75CC9875BB
:106520009853C298C299D2ACC2BC75C8347599064A
:106530002275C800C2ACC2AD75980075CC2B75CD64
:10654000EBD2AD75C8042275C800C2ACC2AD759857
:1065500000E58A242BF5CC540F658C24EBF5CDD2C5
:10656000AD75C804227580FF7590FF75A0FF758F0B
:1065700001120886D228D2A0755700755800C23A79
:10658000A23AB3920AC23BA23BB3920BC23CA23CDA
:10659000B3920CE4F542783D75F010F2D5F0FCC2F0
:1065A00071C272C273C274C237C238C239C259C210
:1065B0005BC25CC25D755401755500C260D264C295
:1065C00065D26AC226C21CC21DC21EC21FC246C2FA
:1065D00020C221756D01C22AC22B755010E4F54905
:1065E000F54AF54BF535F537751E00751F80753F7B
:1065F00007754000E4F552F55AF559F562F563F573
:106600004575440F75460F751D0474377836F2785A
:1066100037F27838F2D231D232D233755103755312
:106620000178A87A0576FF08DAFBC21A7820E47AA6
:1066300007F208DAFCC21B755CFF855C5EC222C2F1
:1066400013C248756F1E757100C27AC218C219C292
:1066500014C215C216C276C277121A147556FAB24F
:10666000031218187533FF7534FF757800D27B75E7
:106670007B00782F740AF2D20F758901758A3E75F6
:106680008C5DC2B9D2A9D28CD2B612650CD2AFD26F
:10669000B4C293D2B3B20312181822C2AF020000E0
:1066A000D6435243206C696E6961203300D7435250
:1066B00044206C696E6961203400C2AF7556FAB22D
:1066C00003121818120483B203121818120483B2AA
:1066D00003121818D2A07581CD75D000126565120D
:1066E0005E89C0E0EAC0E0C083C082900069126A9F
:1066F000CAD082D083D0E0AAE0D0E0125C971262C8
:106700006912223E7556FA12111E755B031232E1B0
:10671000120552751880751903751A6A12178FD2EF
:106720002930130F120FAA125D99125DE9125B480E
:106730001261E6D2A0D2AFC228C22900000020A078
:106740000912048320A00302225830131530480395
:10675000120FAA30130C125D99125DE9125B4812F8
:1067600061E6E5716003D5710512593C800CC206E3
:10677000C26BD208D26DC207C26CE56F700630479B
:1067800003125C69C26EC208C26D1261D1C276C2C8
:1067900077D2701227002067052066028030303FD4
:1067A00022305C1F125E89C0E0EAC0E0C083C08274
:1067B00090042D126ACAD082D083D0E0AAE0D0E043
:1067C0000267C61238A5782FE215E0F27008782F1C
:1067D0007414F20267330267530074A212686EE801
:1067E0001268A9E91268A91268E02274A212686E00
:1067F000E81268A9E71268A909D582F81268E022B0
:1068000074A212686EE81268A974A312686E126806
:10681000C9F709D582041268E022C296D297000017
:1068200000C29780E974A212686EE81268A9126823
:10683000322274A312686E1268C9F91268E02274D9
:10684000A27A08C296000000C297335005D2960281
:106850006854C296D297000000C297DAEDD2960033
:10686000D297000000309604C297C322D3227A0840
:10687000D296D29700000000000000000000000047
:1068800000000000C296000000C297335005D29667
:10689000026895C296D297000000C297DAEDD296B0
:1068A00000D297000000C297227A08335005D29692
:1068B0000268B5C296D297000000C297DAEDD29670
:1068C00000D297000000C297227A08D296C29700A1
:1068D000000000D297C3309601B333DAF0C297229A
:1068E000C296000000D297000000D29622787C76F3
:1068F000000876007880E6543FF67800797CC08204
:106900007582071267EBD08212046B227802797EBF
:10691000C082758205126800D082227882E603C4A4
:10692000540775F018A4C0E07880E6C4540375F0ED
:106930000AA4F5F0E6540F25F0D0F025F075F03CF0
:10694000A4C0F0C0E0787FE6C4540775F00AA4F54F
:10695000F0E6540F25F0D0F025F0F5F0D0E034004B
:10696000C5F022000000000022C2ABC28E53890F86
:10697000438910758B60758DFFC28FD28E308FFD6D
:10698000C28E22C201B203121818B20312181812D2
:106990000483B203121818120483B20312181812D7
:1069A0000483B2031218181204837438F580D2A736
:1069B000126963C2A7B2031218181204837438F55F
:1069C00080D2A7126963C2A7B203121818120483F7
:1069D0007438F580D2A7126963C2A7126969126977
:1069E000697438F580D2A7126963C2A71269697405
:1069F00008F580D2A7126963C2A71269697401F50C
:106A000080D2A7126963C2A71269697406F580D2A1
:106A1000A7126963C2A7B20312181812048322C214
:106A200001B2031218184480F580D2A7126963C21C
:106A3000A712696922C201B203121818547F444098
:106A4000F580D2A7126963C2A712696922D201B286
:106A500003121818126969126969F580D2A71269C0
:106A600063C2A7126969C201B20312181822B4D115
:106A7000087400126A1F026AC9B4D2087440126A0C
:106A80001F026AC9B4D6087480126A1F026AC9B4A8
:106A9000D70874C0126A1F026AC9B4D306126B27E2
:106AA000026AC9B4D41C75F00A20591DC0F075F0F3
:106AB0000F120483120483D5F0F7D0F0D5F0EA0268
:106AC0006AC9906BC093126A4D22EEC0E0EFC0E03D
:106AD0007A00EA0A936037B4D526EA603193602ED3
:106AE00014FFEA05E06027936024FE30130E125E67
:106AF000FF50090A0AEA2E4015FA800F0A0A800B95
:106B0000C083C082126A6ED082D083EA70C5D0E0A2
:106B1000FFD0E0FE22E6600EC083C082126A6ED013
:106B200082D08308DAEF22C201B203121818C083A0
:106B3000C082C0E07401F580D2A7126963C2A7B217
:106B400003121818120483D0E0D082D08322C2012D
:106B5000B203121818C083C082C0E07402F580D25C
:106B6000A7126963C2A7B203121818120483D0E0F7
:106B7000D082D08322C201B20312181854034404F5
:106B8000F580D2A7126963C2A712696922C201B255
:106B90000312181854074408F580D2A7126963122B
:106BA0006963C2A712696922C201B203121818549C
:106BB0000C4410F580D2A7126963C2A7126969223A
:106BC000000102030405060708090A0B0C0D0E0F4D
:106BD0003031323334353637383941424344454613
:106BE000202122232425262728292A2B2C2D2E2F2D
:106BF000303132333435363738393A3B3C3D3E3F1D
:106C0000404142434445464748494A4B4C4D4E4F0C
:106C1000505152535455565758595A5B5C5D5E5FFC
:106C2000606162636465666768696A6B6C6D6E6FEC
:106C3000707172737475767778797A7B7C7D7E7FDC
:106C4000F869706C6C6C086C6C6C6C6C6C096C6CBE
:106C50006C0A0B6C6C6C6C6C6C6C6C6C0D6C0D6CF5
:106C60006C6C0C6C0F6C0F0E6C6C6C6C6C6C6C6CDC
:106C70006C6C0C0B0F6C0F0E6C086C6C6C6C6C0EEF
:106C80006C6C0C6C0F6C0F0E6C6C6C6C6C6C6C6CBC
:106C90006C6C0C6C0F6C0F0E6C6C6C6C6C6C6C6CAC
:106CA0006C6C0C6C0F6C090E6C6C0A6C6C6C6C6C04
:106CB0006C0F0C0C0F6C0F0E6C6C6C6C6C6C6C6C49
:106CC000000E010F110F020002040E1010110E0031
:106CD000000E111F100E02000C0405060C040E001D
:106CE00002040E1111110E0002040E100E011E00FE
:106CF00004001F0204081F000102161911111100DF
:106D000002041F0204081F000E1101020400040007
:106D10007406126B757400126A357E407F00906CA9
:106D2000C0EF0F93126A4DDEF522C083C082740655
:106D3000126B757438126A357E087F00D082D0835A
:106D4000C083C082EF0F93126A4DDEF0D082D083F1
:106D50002200000000000000000000000000000011
:106D60000000000000000000000000000000000023
:106D70000000000000000000000000000000000013
:106D80000000000000000000000000000000000003
:106D900000000000000000000000000000000000F3
:106FC000000000000000000000000000000050521F
:106FD0003330324C434420763130362E35204864ED
:106FE000773A462034303030752032392D30332D09
:106FF00030342031383A323020204352433D00169D
:00000001FF
:0300000306028072
